:100000000C9450070C9476070C9476070C947607A2
:100010000C9476070C9476070C9476070C9476076C
:100020000C9476070C9476070C9433480C944E4845
:100030000C9476070C9476070C9476070C9476074C
:100040000C9476070C9476070C9476070C9476073C
:100050000C9476070C9476070C9476070C9476072C
:100060000C9476070C9476070C9476070C9476071C
:100070000C9476070C9476070C9476070C9476070C
:100080000C9476070C9476070C9476070C947607FC
:100090000C9476070C9476070C9476070C94354AEA
:1000A0000C946F4A0C94A94A0C94E34A0C9476077A
:1000B0000C9476070C9476070C9476070C947607CC
:1000C0000C9476070C9476070C9476070C947607BC
:1000D0000C9476070C9476070C9476070C947607AC
:1000E0000C9476070C9476070C9476070C9476079C
:1000F0000C9476070C9476070C9476070C9476078C
:100100000C9476070C9476070C9476070C9476077B
:100110000C9476070C9476070C9476070C944D4952
:100120000C9487490C94C1490C94FB490C947607B4
:100130000C9476070C9476070C9476070C9476074B
:100140000C9476070C9476070C9476070C9476073B
:100150000C9476070C9476070C9476070C9476072B
:100160000C9476070C9476070C9476070C9476071B
:100170000C9476070C9476070C9476070C9476070B
:100180000C9476070C9476070C9476070C947607FB
:100190000C9476070C9476070C9476070C947607EB
:1001A0000C9476070C9476070C9476070C947607DB
:1001B0000C9476070C9476070C9476070C947607CB
:1001C0000C9476070C9476070C9476070C947607BB
:1001D0000C9476070C9476070C9476070C947607AB
:1001E0000C9476070C9476070C9476070C9476079B
:1001F0000C947607485454502F312E302032303032
:10020000204F4B0A5365727665723A20776C705FA7
:1002100068747470640A436F6E74656E742D7479BB
:1002200070653A20696D6167652F6769660A0A0023
:1002300047494638396145017B00A10000FFFFFFB7
:10024000006699000000FFFFFF21FE114372656107
:1002500074656420776974682047494D50002C000C
:1002600000000045017B000002FE848FA9CBED0F4A
:10027000A39CB4DA8BB3DEBCFB0F86E24896E6891A
:10028000A6EACAB6EE0BC7F24CD7F68DE7FACEF760
:10029000FE0F0C0A87C4A2F1884C2A97CCA6F3095A
:1002A0008D4AA7D4AAF58A6505B6DCAEF70B0E8B8E
:1002B000C76471F60C2DABD7EC36190D3FBAE7F4D5
:1002C000FA3B8EFFD9F77C7BFE9FD32738C80668A0
:1002D000384398A81876D8D8B2081919E048792276
:1002E00079A958A92982D929B809DAE139CA176A3E
:1002F0008A419A4A77CA3AA1FAEAD62AEB005BAB5E
:10030000368BAB60BB6B96EB0BC01BECF5EB2B6C31
:10031000BC458C7B6C9C3CBB2CDC2CFB1C1CDD3A58
:10032000CD5BCD7ABD9B7DBA6DDB6DFA5D1B1E3A50
:100330000E5B0E7AFE9ABEB9AEDAAEF99E1A5F393E
:100340004F5A4F793F9AEFB8EFD9AFD1BF4E010F57
:100350000DC454D0D0C14B09012D94D4F0CFC34863
:1003600011F34C845411CF1DFE5D601A8CF158A618
:10037000421B04024A9A14B0E0E4C9942A511E6850
:10038000290366B88D091831B0F980A6AB5B2465E6
:10039000F6F4F9122800A12D8836D3790027C76119
:1003A000123E5EE01954A5829625A70A35BA022BA3
:1003B00031A40694D664DAB4D7539D5413503569EA
:1003C000F6AAD4185A7F7105D6F126D8B0715139E2
:1003D0008DBAF26759BD68F9BA84D1B6D8DDAF5F7E
:1003E0004072913B6969E10C64D59E4DBB7647E054
:1003F0005C6FBD22987B199962CC490FD3128BB7E1
:10040000AF81B355FDFA98AC6C70E6C50B58AFDE02
:10041000CCB96B6CD996F70E255DFA76E4D07F47A0
:10042000FBCCCB127883C9A879E77EF0B847E5BA50
:10043000B05B2726CC7C7517C4D17503C79DDB360E
:100440006FC82B8962EFCDFD7878ED56B10FFFCEE6
:10045000E3ADC8D9CE414BF7DCDEB5EFC8E8E70B1A
:10046000B72FBE2CD0EFF7FEF183F78F5B70FC95B2
:10047000376020AAD9C5DE7BD5D1361D75B1FD66A2
:100480001E8004E6572080018E2760851692365E16
:100490008438A847C182D0B9D7197B245A87964C93
:1004A0002AEEB69D5FDAF1C7228AFFC1789F63C248
:1004B000D9289A0D20EE045F4E21C5D7E3880D762A
:1004C00028A37F32FE57A48B10C6481E8EE21D69FA
:1004D000DA04C5DDB0235DCF41009F8822C2B5A0FC
:1004E0007E6BC1449E914A228995931866D85B9889
:1004F000E7C5E84395110489E0950ACA39A7661D46
:10050000DAA6618BC62179248C51EE59619E63F67F
:10051000F7E1810C0EB91407B36D79629F377A78D1
:10052000E69E0CD0B81F8B94EE46239A1CEAB09C32
:100530007C9921C6239D87DA091B9C1BE658DF8422
:10054000E0A9792AA44E663A289BB016DAA8659DE0
:1005500001F926A2733A385BAA8EE6F8A784935E67
:100560008AAAA5C43EF9FE2BA1C9024B43A7268A3D
:10057000EAA990BC1A2622A4AD0E5BA356AC3A6041
:10058000A6079B22F76D0DCEEAFA2990A46E469D30
:100590008FB69EAA2A9B491AB7A6B2DC1AEB6E0642
:1005A00053BEABA3A15C3E6B188F1BE8FB6BBBCCAF
:1005B000EA29ACA6AB762BA98B146CABAA81B53219
:1005C0002A2A63115BB9E58583C64B61BDCB7AC727
:1005D00024B109EB991CC1E2EABB2E971E984A711F
:1005E000C521DFC927BE50622C28C794B21CAEC7F4
:1005F000B4AE5B32B916E89CAB7AE18E093391F365
:10060000FAD9B0C02BB7FAAAC554920C31CAEDBDC5
:1006100037D68FD8BAFB73B02F83AB74A4460F0CB8
:1006200028D5828EFC70B4A34EBC6F8309960AF065
:10063000D59A0E0D2CC345B38DACD0111C0D73CBC8
:10064000F95E94484671E09D89DE68F09DB7DF67EA
:10065000004E88E08313FE89E158209EB8E25630B0
:10066000DE87E35740AD5E8AE45550BE87E5976369
:100670005E87E65470DEB9E75280BE8AE851903E4C
:1006800087E9A7A33E92EA4FB0DEBAEB4DC05E8881
:10069000ECB3D30E95ED4AE09EBBEE48F02EB5EFDD
:1006A000BF039FB6F040105FBCF16D225FB2F27ADB
:1006B00030BFA5F3CB437FB6F43B505FBDF59C62E2
:1006C000EFB4F6CA714FB6F7D7832F3E11E4976F98
:1006D0003EF6E8A74FFDFAEC23EF7E11CCC72F3F83
:1006E000F1F41B01FCFDC3B3AE7F12A4F77F3BC640
:1006F00001F0730719A0010F88C0042A70810C6CE7
:10070000A0031F08C1084A708214ACA0052F8841BD
:10071000CD1500003B485454502F312E302034303A
:10072000342046696C65206E6F7420666F756E6448
:100730000A5365727665723A20776C705F687474DC
:1007400070640A436F6E74656E742D747970653AC7
:1007500020746578742F68746D6C0A0A3C68746D37
:100760006C3E3C686561643E3C7469746C653E6FC8
:10077000574C207069636F2048545450205765626D
:10078000207365727665723C2F7469746C653E3CAB
:100790002F686561643E3C626F64793E3C68323E1E
:1007A000343034202D2050616765206E6F742066D0
:1007B0006F756E643C2F68323E3C703E536F7272B0
:1007C000792C20746865207061676520796F7520C9
:1007D0006172652072657175657374696E672077E3
:1007E0006173206E6F7420666F756E64206F6E206B
:1007F00074686973207365727665722E3C2F703E43
:100800003C2F626F64793E3C2F68746D6C3E0048EB
:100810005454502F312E3020323030204F4B0A5359
:1008200065727665723A20776C705F687474706474
:100830000A436F6E74656E742D747970653A207416
:100840006578742F68746D6C0A0A3C21444F4354D8
:100850005950452048544D4C205055424C49432056
:10086000222D2F2F5733432F2F4454442048544DCB
:100870004C20342E3031205472616E736974696F6C
:100880006E616C2F2F454E222022687474703A2FAF
:100890002F7777772E77332E6F72672F54522F680A
:1008A000746D6C342F6C6F6F73652E647464223EAC
:1008B0003C68746D6C3E3C686561643E3C74697470
:1008C0006C653E6F574C207069636F2048545450DC
:1008D00020576562207365727665723C2F74697467
:1008E0006C653E3C2F686561643E3C626F647920B4
:1008F0007374796C653D666F6E742D66616D696C9D
:10090000793A617269616C3E3C7461626C653E3C2F
:1009100074723E3C74642077696474683D2231309F
:1009200030223E3C2F74643E3C74643E3C746162F1
:100930006C653E3C74722076616C69676E3D227412
:100940006F70223E3C74643E3C696D672073726335
:100950003D226C6F676F2E6769662220616C743D63
:10096000226C6F676F227469746C653D226C6F67CF
:100970006F223E3C2F74643E3C2F74723E3C747276
:100980003E3C74642077696474683D2235303022BF
:100990003E3C68323E576562205365727665722030
:1009A00072756E6E696E67206F6E206F574C207087
:1009B00069636F3C2F68323E3C703E546865207717
:1009C0006562207061676520697320736572766562
:1009D0006420627920776C705F687474706420752D
:1009E00073696E6720746865205350423830302038
:1009F000574C414E206D6F64756C6520616E6420AC
:100A0000746865206F574C2D7069636F26636F7033
:100A1000793B20536F667477617265204150493B82
:100A2000206120756E697175652057692D466920B2
:100A3000736F6C7574696F6E2066726F6D203C62A7
:100A40003E4826616D703B4420576972656C657342
:100A5000732041423C2F623E2E3C2F703E3C687218
:100A60003E3C7461626C653E003C74723E3C746452
:100A70003E495020416464726573733A20003C2FF4
:100A800074643E3C74643E3C623E3C2F623E3C2FAC
:100A900074643E3C2F74723E003C74723E3C74643D
:100AA0003E4D414320416464726573733A20003CBB
:100AB0002F74643E3C74643E3C623E3C2F623E3C7C
:100AC0002F74643E3C2F74723E003C74723E3C7442
:100AD000643E3C666F726D206D6574686F643D2284
:100AE0006765742220616374696F6E3D22223E3C0B
:100AF000703E3C696E70757420747970653D227328
:100B000075626D697422207374796C653D22686525
:100B1000696768743A2035307078222076616C7588
:100B2000653D2252656672657368223E3C2F703EB9
:100B30003C2F666F726D3E3C2F74643E3C2F747286
:100B40003E3C2F7461626C653E3C62723E3C666F57
:100B5000726D2069643D22666F726D226E616D65F3
:100B60003D22666F726D22206D6574686F643D2250
:100B70006765742220616374696F6E3D22696E64DB
:100B800065782E68746D6C223E3C6669656C647392
:100B900065743E3C6C6567656E643E4C45442063FD
:100BA0006F6E74726F6C3C2F6C6567656E643E3C53
:100BB000696E70757420747970653D227375626D0D
:100BC000697422207374796C653D22686569676871
:100BD000743A203530707822206E616D653D227444
:100BE0006F67676C65222076616C75653D224C45A8
:100BF0004430223E266E627370266E6273703C69CA
:100C00006E70757420747970653D227375626D69BC
:100C10007422207374796C653D2268656967687415
:100C20003A203530707822206E616D653D22746FF8
:100C300067676C65222076616C75653D224C454482
:100C400031223E266E627370266E6273703C696E4E
:100C500070757420747970653D227375626D697466
:100C600022207374796C653D226865696768743AFF
:100C7000203530707822206E616D653D22746F677B
:100C8000676C65222076616C75653D224C45443267
:100C9000223E266E627370266E6273703C696E70BF
:100CA000757420747970653D227375626D69742264
:100CB000207374796C653D226865696768743A20B1
:100CC0003530707822206E616D653D22746F6767E4
:100CD0006C65222076616C75653D224C454433225B
:100CE0003E266E627370266E6273703C703E003CEE
:100CF000696E70757420747970653D227375626DCC
:100D0000697422207374796C653D2268656967682F
:100D1000743A203530707822206E616D653D227402
:100D20006F67676C65222076616C75653D224C4566
:100D30004434223E266E627370266E6273703C6984
:100D40006E70757420747970653D227375626D697B
:100D50007422207374796C653D22686569676874D4
:100D60003A203530707822206E616D653D22746FB7
:100D700067676C65222076616C75653D224C454441
:100D800035223E266E627370266E6273703C696E09
:100D900070757420747970653D227375626D697425
:100DA00022207374796C653D226865696768743ABE
:100DB000203530707822206E616D653D22746F673A
:100DC000676C65222076616C75653D224C45443622
:100DD000223E266E627370266E6273703C696E707E
:100DE000757420747970653D227375626D69742223
:100DF000207374796C653D226865696768743A2070
:100E00003530707822206E616D653D22746F6767A2
:100E10006C65222076616C75653D224C4544372215
:100E20003E266E627370266E6273703C2F66696533
:100E30006C647365743E3C2F666F726D3E3C2F741C
:100E4000643E3C74643E266E6273703B3C2F746457
:100E50003E3C2F74723E3C2F7461626C653E3C2FA9
:100E600074643E3C74642077696474683D22323057
:100E700025223E3C2F74643E3C2F74723E3C2F74FE
:100E800061626C653E3C2F626F64793E3C2F6874F2
:100E90006D6C3E006364696E6F70737578585B00AB
:100EA00011241FBECFEFDFE3DEBFCDBF00E00CBFDC
:100EB00018BE19BE1ABE1BBE13E3A0E0B0E2E4E9FF
:100EC000F7EB00E00BBF02C007900D92AE32B10706
:100ED000D9F71BBE14E3AEE2B3E301C01D92A13209
:100EE000B107E1F70E94C4420C94C85B0C94000067
:100EF0009BB78BBFFB018091CA014093CA017DE97A
:100F000070933400E8958093CA019BBF08952091A7
:100F1000CF0127FDFCCF9BB78BBFFB018091CA019E
:100F200023E22093CA010A01E89511248093CA01A3
:100F30009BBF0895E0913033F09131330BC0228193
:100F400022FD05C0208131812817390729F003804F
:100F5000F481E02D309799F7CF0108959C01AB0102
:100F6000A0913233B0913333ED91FC9111971696E5
:100F70008D919C911797B901199508959C01AB012A
:100F8000A0913233B09133331296ED91FC911397C7
:100F900016968D919C911797B90119950895A09176
:100FA0003233B09133331496ED91FC91159730970D
:100FB00039F016968D919C91179761E070E0199524
:100FC0000895A0913233B09133331496ED91FC9192
:100FD0001597309739F016968D919C91179760E090
:100FE00070E019950895E0913233F09133338089A0
:100FF00083FD0CC008951C96ED91FC911D973097D0
:1010000049F01E968D919C911F971995A0913233AE
:10101000B091333351968C915197882361F3519657
:101020001C9251970895AF92BF92CF92DF92EF92A8
:10103000FF920F931F93CF93DF937C015B01EA0133
:101040006901289688E090E0C80ED91ECE010E9462
:101050007414F701808391831282A3821482158213
:1010600016820115110579F00E94CF07C701BE0154
:101070000E94BE070E94F307C701B6010E94AE0797
:101080000E94E1070AC0C701BE010E94BE070E947C
:10109000F307C701B6010E94AE07F7018081918175
:1010A0000E947814F70180839183848195810E9446
:1010B00078149C01F70184839583808191818C153C
:1010C0009D0541F48281813029F4838190E08A1565
:1010D0009B0511F020EF3FEFC901DF91CF911F91E8
:1010E0000F91FF90EF90DF90CF90BF90AF90089559
:1010F000CF92DF92EF92FF920F931F93CF93DF93E4
:101100007C016B01EA018901E0913233F0913333C4
:10111000208531852115310531F08285938561E087
:1011200070E0F9011995C701B601AE01980101E01F
:1011300010E00E941308082FC92FA0913233B091FC
:1011400033331896ED91FC911997309739F01A9630
:101150008D919C911B9760E070E01995802F9C2FDA
:10116000DF91CF911F910F91FF90EF90DF90CF9083
:1011700008954F925F926F927F928F929F92AF925B
:10118000BF92CF92DF92EF92FF920F931F93CF9374
:10119000DF93EC015B014A013901280100913233F0
:1011A00010913333C801829669E070E040E050E06E
:1011B00028E130E00E947808209749F0F80142A524
:1011C00053A564A575A5488359836A837B83A114BD
:1011D000B10451F0F80146A557A560A971A9F50120
:1011E00040835183628373838114910451F0F80129
:1011F00042A953A964A975A9F4014083518362836C
:1012000073836114710451F0F80146A957A960ADC8
:1012100071ADF301408351836283738341145104A0
:1012200041F0F80127AD332727FD3095F2012083E7
:101230003183C114D10441F0F80126AD332727FDD5
:101240003095F60120833183E114F10451F0F80167
:1012500042AD53AD64AD75ADF701408351836283F8
:101260007383DF91CF911F910F91FF90EF90DF90EB
:10127000CF90BF90AF909F908F907F906F905F9036
:101280004F9008950F93CF93DF93E0913233F09115
:101290003333009751F0EC0188819981AA81BB8199
:1012A00082A793A7A4A7B5A704C012A613A614A645
:1012B00015A66115710551F0EB0188819981AA810C
:1012C000BB8186A797A7A0ABB1AB04C016A617A693
:1012D00010AA11AA4115510551F0EA01888199819E
:1012E000AA81BB8182AB93ABA4ABB5AB04C012AAFD
:1012F00013AA14AA15AA2115310551F0E901888114
:101300009981AA81BB8186AB97ABA0AFB1AF04C076
:1013100016AA17AA10AE11AE02AFCF01829668E0EE
:1013200070E044E150E020E030E00E947808DF9176
:10133000CF910F910895CF92DF92EF92FF920F938A
:101340001F93CF93DF936C01EB0100913233109127
:101350003333209709F454C0CB0183709070009709
:1013600029F0862F837024E0281B01C020E082E250
:10137000E82EF12CE00EF11EF80120A7CE01089610
:10138000820F911D0E947414F80182A393A382E03E
:1013900084A38BE185A316A217A2C70168E070E0C1
:1013A0000E94BE07F80180A5C80FD11DC601BE016D
:1013B0000E94BE078C179D0731F50E94F307C701F5
:1013C00068E070E00E94AE07F80182A193A10E943C
:1013D0007814F80182A393A386A197A10E947814A0
:1013E0009C01F80186A397A382A193A1883091055F
:1013F00051F484A1833039F485A18B3131F003C0DD
:1014000020E030E002C020EF3FEFC901DF91CF9133
:101410001F910F91FF90EF90DF90CF9008958F92E2
:101420009F92AF92BF92CF92DF92EF92FF920F9373
:101430001F93CF93DF930F92CDB7DEB74C016B01B3
:101440005A01790187E7898381E693E380933233F8
:101450009093333360E070E042EB50E00E94AD16B1
:10146000E0913233F0913333C082D182A282B382D1
:10147000E482F5820683178381E08816910421F4C3
:1014800080898860808B1DC00E94CF078E010F5F0E
:101490001F4FC80161E070E00E94BE07C80161E013
:1014A00070E00E94AE07E02E012F06C08E2D902F17
:1014B00061E070E00E94AE0789818E32B9F30E942C
:1014C000E10780E090E00F90DF91CF911F910F91A5
:1014D000FF90EF90DF90CF90BF90AF909F908F9054
:1014E00008950F931F93CF93DF938C01C0913233F4
:1014F000D0913333CE01829663E270E040E050E059
:1015000024E030E00E94780897FD05C08AA5F80124
:10151000808380E090E0DF91CF911F910F9108953B
:10152000EF92FF920F931F93CF93DF93EC018B0108
:10153000E0913233F0913333009719F081E082A7C4
:1015400001C012A6CF0182966FE170E044E050E046
:1015500020E030E00E9478087C01E0913233F09185
:101560003333C087D18702871387C80160E070E0FA
:10157000FE011995C701DF91CF911F910F91FF9047
:10158000EF900895E0913233F0913333848795875B
:10159000668777870895E0913233F091333381E0A5
:1015A000818B08950F931F93CF93DF930F92CDB745
:1015B000DEB7009132331091333349830E947C149B
:1015C000DC01CB01F80182A793A7A4A7B5A74981A5
:1015D00046A78091323390913333829660E070E079
:1015E00048E050E024E030E00E9478080F90DF915E
:1015F000CF911F910F910895BF92CF92DF92EF92FA
:10160000FF920F931F93CF93DF930F920F92CDB75B
:10161000DEB787E78A83A0913233B09133331896CF
:10162000ED91FC911997309739F01A968D919C9114
:101630001B9761E070E019958091323390913333BC
:10164000829668E170E040E050E020E030E00E94E7
:1016500078086C0197FD35C0E0913233F091333357
:10166000808983FD2EC00E94CF078E010E5F1F4F21
:10167000C80161E070E00E94BE077E010894E11C91
:10168000F11CC70161E070E00E94AE07B02E0F2D83
:101690000CC08B2D912F61E070E00E94BE078E2D53
:1016A000902F61E070E00E94AE078981873789F74B
:1016B0000E94E107E0913233F091333380898F7ECD
:1016C000808BA0913233B09133331896ED91FC9119
:1016D0001997309739F01A968D919C911B9760E07D
:1016E00070E01995C6010F900F90DF91CF911F9177
:1016F0000F91FF90EF90DF90CF90BF9008956F9281
:101700007F928F929F92AF92BF92CF92DF92EF9291
:10171000FF920F931F93CF93DF933C017B016A01EC
:101720004901C0913233D0913333CE01829662E0C9
:1017300070E040E050E024E230E00E9478085C0174
:1017400097FD3AC08AA590E0A0E0B0E0BC01552723
:1017500044278CA590E0A0E0B0E0482B592B6A2BE1
:101760007B2B8BA590E0A0E0B0E0BA2FA92F982F9B
:101770008827482B592B6A2B7B2BF30140835183FD
:1017800062837383E114F10451F0C114D10439F080
:10179000BE01625D7F4FC701A6010E94BC16811485
:1017A000910451F00115110539F0BE01625C7F4FC3
:1017B000C401A8010E94BC16C501DF91CF911F9101
:1017C0000F91FF90EF90DF90CF90BF90AF909F90E0
:1017D0008F907F906F900895E0913233F091333382
:1017E000828B938B648B758B089586EF9FEF0895A2
:1017F00086EF9FEF0895AF92BF92CF92DF92EF9264
:10180000FF920F931F93CF93DF938C016B015A01CB
:10181000E0903233F0903333E701AA96CE0160E0D6
:1018200070E048E650E00E94AD160115110531F058
:10183000CE01B80141E250E00E94AA16C114D104C1
:1018400061F081E0A816B10439F1C6010E94B31617
:1018500008978833910500F112C0F701E257FF4F56
:10186000A0828091323390913333829663E070E0AE
:1018700048E650E020E030E00E94780802C08EEF99
:101880009FEFDF91CF911F910F91FF90EF90DF902D
:10189000CF90BF90AF900895C701825B9F4FB60174
:1018A0004FE350E00E94BC16D8CF80913233909124
:1018B0003333829664E070E040E050E020E030E0B6
:1018C0000E94780808950F931F9300E010E00E9493
:1018D00042091F910F910895CF92DF92EF92FF92EC
:1018E0000F931F9300E010E0EE24FF24CC24DD24AE
:1018F0000E94B9081F910F91FF90EF90DF90CF9059
:1019000008950F931F938C0180E090E060E070E0F9
:1019100040E050E020E030E00E9442091F910F912A
:101920000895CF92DF92EF92FF920F931F938C0155
:1019300080E090E060E070E040E050E020E030E0E7
:10194000EE24FF24CC24DD240E94B9081F910F91BE
:10195000FF90EF90DF90CF900895E0913233F091B7
:10196000333382A7CF01829669E170E044E050E012
:1019700020E030E00E9478080895E0913233F09141
:101980003333868B978B608F718F08950F931F93DE
:10199000CF93DF938C01C0913233D09133330097D2
:1019A000D9F0CE01829666E070E040E050E024E39A
:1019B00030E00E94780897FF04C02FEF8C3F920719
:1019C00069F4BE01665D7F4FC80146E050E00E94A9
:1019D000AA1680E090E002C08EEF9FEFDF91CF91DA
:1019E0001F910F9108950F931F93CF93DF93EC01F5
:1019F00000913233109133330097B9F1C8018296C8
:101A000066E070E040E050E024E330E00E947808B7
:101A100097FD2DC0B801605D7F4FCE01819646E0F5
:101A200050E00E94AA16B8016A5C7F4FCE0141E2E5
:101A300050E00E94AA16F801E65AFF4F808191817A
:101A40000E9478148FA398A7F801E45AFF4F808171
:101A500091810E94781489A79AA71DA61BA61CA68F
:101A60001EA61FA680E090E002C08EEF9FEFDF91E0
:101A7000CF911F910F910895CF92DF92EF92FF9235
:101A80000F931F93CF93DF930F92CDB7DEB7F82E4E
:101A9000C0903233D09033338FE090E069830E945E
:101AA00086168C016981009779F1F601F2A663A789
:101AB000809132339091333382966BE070E044E052
:101AC00050E020E030E00E9478087C0197FF04C0DD
:101AD000C8010E94A7161CC0F8018083918313825D
:101AE0001482E0913033F0913133309731F4009328
:101AF0003033109331330CC0FC0183819481009703
:101B0000D9F70383148304C04DEFE42E4FEFF42E76
:101B1000C7010F90DF91CF911F910F91FF90EF9030
:101B2000DF90CF9008950F931F93CF93DF938B0196
:101B3000EA010E949A07FC01009739F00783108799
:101B4000C387D48780E090E002C08EEF9FEFDF91E3
:101B5000CF911F910F9108950F931F93CF93DF9310
:101B60008B01EA010E949A07FC01009739F0018776
:101B70001287C587D68780E090E002C08EEF9FEF86
:101B8000DF91CF911F910F910895EF92FF920F93E4
:101B90001F93CF93DF93EB017A01009132331091C1
:101BA00033330E947414F80186A797A7888199811E
:101BB000AA81BB8182A793A7A4A7B5A7C7010E944A
:101BC0007414F80180AB91AB809132339091333330
:101BD00082966CE070E048E050E020E030E00E9447
:101BE0007808DF91CF911F910F91FF90EF900895AA
:101BF000AF92BF92CF92DF92FF920F931F93CF933A
:101C0000DF938C01F62E5A016901C0913233D091D5
:101C100033330E949A07FC010097C9F0A582B6826F
:101C2000C386D4861282C8010E9474148AA79BA717
:101C3000FCA6809132339091333382966DE070E050
:101C400044E050E020E030E00E94780802C08EEFCF
:101C50009FEFDF91CF911F910F91FF90DF90CF9079
:101C6000BF90AF900895CF92DF92EF92FF920F93C3
:101C70001F93CF93DF937C01EB016A010091323314
:101C8000109133330E949A07009721F1FC011282D0
:101C9000C7010E947414F80186A797A788819981CB
:101CA000AA81BB8182A793A7A4A7B5A7C6010E945A
:101CB0007414F80180AB91AB80913233909133333F
:101CC00082966EE070E048E050E020E030E00E9454
:101CD000780802C08EEF9FEFDF91CF911F910F9197
:101CE000FF90EF90DF90CF900895EF92FF920F93C7
:101CF0001F93CF93DF937C01C0913233D091333364
:101D00008FE090E00E9486168C01009771F1C70168
:101D10000E9474148AA79BA7809132339091333329
:101D2000829664E170E044E050E020E030E00E9400
:101D30007808EC0197FF04C0C8010E94A71617C0DD
:101D4000F80180839183138214828281816082836F
:101D5000E0913033F091313301C0FC0183819481F3
:101D60000097D9F70383148302C0CDEFDFEFCE01D4
:101D7000DF91CF911F910F91FF90EF9008950F93F6
:101D80001F93CF93DF938C01C0913233D0913333C3
:101D90000E9474148AA79BA78091323390913333A9
:101DA00082966FE070E044E050E020E030E00E9476
:101DB00078082091303330913133F901C0E0D0E020
:101DC0002DC0808191818017910719F5828182FD54
:101DD00020C0A0913233B091333350969C915097EC
:101DE00092FF03C0846082831BC0209751F4D90105
:101DF00013968D919C911497809330339093313347
:101E000004C0838194818B839C83CF010E94A71699
:101E100007C093818481EF01E92FF82F309789F66D
:101E200080E090E0DF91CF911F910F9108958F9204
:101E30009F92AF92BF92CF92DF92EF92FF920F9359
:101E40001F93CF93DF9300D0CDB7DEB74B017A015C
:101E500000913233109133330E947414F80182A739
:101E600093A7C7010E947414F80184A795A7A091B5
:101E70003233B09133331896ED91FC911997309726
:101E800039F01A968D919C911B9761E070E019953D
:101E90000E94CF078091323390913333829660E174
:101EA00070E044E050E020E030E000E010E00E940C
:101EB00013085C0197FD4DC0E816F9060CF445C007
:101EC000C0903233D09033330097C1F10E94F307B2
:101ED000C601829668E070E00E94AE078C01F601B0
:101EE00082A193A10E947814F60182A393A30830E3
:101EF000110539F524A1243021F525A12B3109F54F
:101F000020A568EFE62E6FEFF62EE21AF108E80E34
:101F1000F91EEA14FB04A9F4C401B7010E94AE073C
:101F20008C018E159F0569F4F60160A5662359F0B2
:101F3000CE01019670E00E94AE0705C000E010E0FF
:101F400002C000EF1FEF580104C050EFA52E5FEF55
:101F5000B52E0E94E107A0913233B0913333189629
:101F6000ED91FC911997309739F01A968D919C91CB
:101F70001B9760E070E01995C5012396CDBFDEBFC9
:101F8000DF91CF911F910F91FF90EF90DF90CF9055
:101F9000BF90AF909F908F900895CF92DF92EF9275
:101FA000FF920F931F93CF93DF936B017A01C09140
:101FB0003233D09133330E9474148AA79BA7C70190
:101FC0000E9474148CA79DA7A0913233B091333333
:101FD0001896ED91FC911997309739F01A968D91DA
:101FE0009C911B9761E070E019950E94CF0780914A
:101FF000323390913333829661E170E044E050E0F7
:1020000020E030E000E010E00E941308EC0197FDB2
:102010000BC0E816F90634F0C601BE010E949B0908
:10202000EC0102C0C0EFDFEF0E94E107A091323364
:10203000B09133331896ED91FC911997309739F0A0
:102040001A968D919C911B9760E070E01995CE01D6
:10205000DF91CF911F910F91FF90EF90DF90CF9084
:102060000895AF92BF92CF92DF92EF92FF920F93BB
:102070001F93CF93DF935B016A01E901780100911F
:102080003233109133330E947414F80186A797A756
:10209000C6010E947414F80180AB91AB88819981CC
:1020A000AA81BB8182A793A7A4A7B5A7C7010E9455
:1020B0007414F80182AB93ABA0913233B0913333F7
:1020C0001896ED91FC911997309739F01A968D91E9
:1020D0009C911B9761E070E019950E94CF07809159
:1020E000323390913333829662E170E04CE050E0FD
:1020F00020E030E000E010E00E941308EC0197FDC2
:102100000BC0C816D90634F0C501BE010E949B0958
:10211000EC0102C0C0EFDFEF0E94E107A091323373
:10212000B09133331896ED91FC911997309739F0AF
:102130001A968D919C911B9760E070E01995CE01E5
:10214000DF91CF911F910F91FF90EF90DF90CF9093
:10215000BF90AF9008950F931F93CF93DF938B01A0
:10216000C0913233D09133330E9474148AA79BA755
:102170008091323390913333829665E170E044E090
:1021800050E024E030E00E94780897FD09C04AA59D
:102190005BA56CA57DA5F8014083518362837383A1
:1021A000DF91CF911F910F910895CF92DF92EF921F
:1021B000FF920F931F93CF93DF93EC017B016A0192
:1021C0000091323310913333009751F10E94B316CE
:1021D0008038910528F5E0913233F0913333828DC8
:1021E000938D009701F5C8018A96BE010E94C5161D
:1021F000809132339091333382966AE070E040E808
:1022000050E020E030E00E94780897FD0EC0E09199
:102210003233F0913333E28EF38EC48ED58E05C007
:102220008EEF9FEF02C082EF9FEFDF91CF911F9162
:102230000F91FF90EF90DF90CF900895CF92DF92B3
:10224000EF92FF920F931F93CF93DF93CDB7DEB73B
:102250002A97CDBFDEBF8091323390913333009700
:1022600009F4DFC1829661E070E040E050E020E0D8
:1022700030E00E947808009709F4D3C1809132338E
:1022800090913333829665E070E040E050E020E0CA
:1022900030E00E9478080097D1F4A0913233B091D9
:1022A00033335296ED91FC915397309761F15096EC
:1022B0008C91509780FD27C0816050968C935097E9
:1022C00054968D919C91559761E070E01BC097FFEB
:1022D0001AC0A0913233B09133335296ED91FC91F4
:1022E0005397309781F050968C91509780FF0BC098
:1022F0008E7F50968C93509754968D919C915597C4
:1023000060E070E01995CE01079660E070E040E073
:1023100050E020E030E000E010E0E3E0EE2EF12CB1
:10232000EC0EFD1E6E010894C11CD11C0E94B90860
:10233000A0913233B09133330097C1F45696ED91AA
:10234000FC915797309759F150968C91509781FD99
:1023500026C0826050968C93509758968D919C9190
:102360005997BE01695F7F4F199519C097FF3EC00D
:102370005696ED91FC9157973097C1F150968C91FC
:10238000509781FF33C08D7F50968C93509758960D
:102390008D919C91599760E070E0199527C0A091AC
:1023A0003233B09133335A96ED91FC915B9730976D
:1023B000E9F089819A81009741F45C968D919C9116
:1023C0005D97BE016D5F7F4F0AC02FEF8F3F920771
:1023D00069F45C968D919C915D9760E070E0199531
:1023E000E0913233F0913333128E138E00913233F9
:1023F00010913333D80150968C91509784FF32C09E
:102400005E968D919C915F97009761F1C8018296CD
:1024100064E270E040E050E024E030E00E947808A0
:1024200097FD03C0F80182A501C080E0A09132337E
:10243000B091333380FF0AC05E96ED91FC915F97B7
:1024400090968D919C91919761E00BC081FF0AC09D
:102450005E96ED91FC915F9790968D919C919197EE
:1024600060E01995E0913233F091333380898460D4
:10247000808B009130331091313393C0D8018D910E
:102480009C910E947414F70182A793A78091323324
:1024900090913333829663E170E044E050E024E0B1
:1024A00030E00E947808AC0197FD22C0D7019A96CF
:1024B0008C919A978130D1F4F801928190FD42C0BD
:1024C0000780F085E02D3097E9F1892F81608D7FBD
:1024D000D80112968C9312976D917C9111971B964F
:1024E0008D919C911C9741E050E057C08430B9F425
:1024F000F801828181FD25C00780F085E02D3097AD
:1025000001F18E7F8260D80112968C9312976D91A3
:102510007C9111971B968D919C911C973CC08330A8
:1025200089F4D8011596ED91FC911697309751F0EA
:102530006D917C9111971B968D919C911C9719958B
:102540002DC084E0141615067CF4D8011996ED917F
:10255000FC911A97309741F06D917C9111971D96DF
:102560008D919C911E9719C08823C1F4F801828136
:1025700080FF14C00184F285E02D309779F08E7FC2
:10258000D80112968C9312976D917C9111971D969C
:102590008D919C911E9740E050E01995F8010381C0
:1025A0001481E0903233F09033330115110509F0B6
:1025B00065CFD70150968C9150978B7F50968C9316
:1025C0005097E0913033F091313300E010E027C0B4
:1025D000828182FF1FC00115110569F4A09130337B
:1025E000B091313313968D919C9114978093303331
:1025F0009093313307C083819481D80113968D93D2
:102600009C931497F380E480CF010E94A716EF2DCE
:10261000FE2D05C0938184818F01E92FF82F30971B
:10262000B9F62A96CDBFDEBFDF91CF911F910F91F2
:10263000FF90EF90DF90CF900895E0913233F091CA
:10264000333382A7CF01829666E170E044E050E028
:1026500020E030E00E94780808950F931F93CF93F5
:10266000DF938C01C0913233D0913333CE01829607
:102670006AE170E040E050E024E030E00E94780839
:1026800097FD03C02AA5F8012083DF91CF911F9108
:102690000F910895E0913233F091333382A7CF0147
:1026A000829667E170E044E050E020E030E00E9474
:1026B0007808089586EF9FEF0895E0913233F09106
:1026C000333321E0009709F420E022A7CF0182965E
:1026D0006EE170E044E050E020E030E00E947808D5
:1026E00008958F929F92AF92BF92CF92DF92EF9216
:1026F000FF920F931F93CF93DF93F82E4A015B0154
:10270000C901B801C0913233D09133330E947C1497
:10271000DC01CB018AA79BA7ACA7BDA7C501B4016B
:102720000E947C14DC01CB018EA79FA7A8ABB9AB9C
:10273000C6010E9474148AAB9BABFCAAEDAA8091DF
:1027400032339091333382966DE170E04FE050E088
:1027500020E030E00E947808DF91CF911F910F9127
:10276000FF90EF90DF90CF90BF90AF909F908F90B1
:102770000895AF92BF92DF92EF92FF920F931F9353
:10278000CF93DF93D82EEB015A01790100913233B8
:1027900010913333C8018A9660E070E048E850E059
:1027A0000E94AD16209749F088819981AA81BB814A
:1027B000F80182A793A7A4A7B5A7C5010E94741426
:1027C000F80186A797A7D0AAE114F10479F0C70110
:1027D0000E94B3168F37910500F5C7010E94B3160A
:1027E000AC01C801C296B7010E94AA16809132338B
:1027F0009091333382966CE170E048E850E020E03D
:1028000030E00E947808009751F4E0913233F09163
:10281000333320892061208B02C08EEF9FEFDF9140
:10282000CF911F910F91FF90EF90DF90BF90AF90ED
:102830000895E0913233F0913333868F978F60A300
:1028400071A380E090E00895E0913233F09133334A
:1028500021E0009709F420E022A7CF01829660E2F0
:1028600070E044E050E020E030E00E9478080895F5
:10287000CF93DF93C0913233D09133330E947C14D5
:10288000DC01CB018AA79BA7ACA7BDA780913233FF
:1028900090913333829661E270E044E050E020E0B2
:1028A00030E00E947808DF91CF910895CF93DF93B5
:1028B000C0913233D09133330E947C14DC01CB01C0
:1028C0008AA79BA7ACA7BDA78091323390913333E1
:1028D000829662E270E044E050E020E030E00E9446
:1028E0007808DF91CF910895982789279827089530
:1028F00098278927982708950F931F93DC01CB0110
:102900000B2F112722273327782F66275527442797
:10291000042B152B262B372B4427582F692F7A2F62
:10292000407050707070042B152B262B372B892F7D
:102930009A2FAB2FBB278070A070B070082B192B7B
:102940002A2B3B2BB801C9011F910F9108950E94BA
:102950007C1408952F923F924F925F926F927F92D4
:102960008F929F92AF92BF92CF92DF92EF92FF929F
:102970000F931F93CF93DF93CDB7DEB76497CDBF8F
:10298000DEBFFC016B8B7C8B0081112707FD10954E
:102990009E01235F3F4F298B3A8B7E010894E11CF7
:1029A000F11C802F80538A3008F03EC1003311059E
:1029B000C1F40181112707FD10950837110541F079
:1029C0000835110529F0319628E0622E712C0CC0D3
:1029D0000281112707FD1095329690E1692E712C26
:1029E00003C08AE0682E712C6F0140E050E0BA010C
:1029F0001301442437FC4094542C902F802F805393
:102A00008A30A0F4CB01BA01A20191010E9440508A
:102A10004B015C01C801C097AC01662757FD60956A
:102A2000762F480D591D6A1D7B1D2AC0B0E16B161B
:102A3000710489F5802F8156863020F0202F215493
:102A4000263048F54A015B01B4E0880C991CAA1CA9
:102A5000BB1CBA95D1F7065F1F4F8A3118F481E687
:102A600090E002C081E490E0F801E81BF90BAF01AF
:102A7000662757FD6095762F482959296A297B29B1
:102A8000D60111960C911197112707FD1095089406
:102A9000C11CD11CB2CFE42F352F0E321105F1F439
:102AA00049895A89E416F50609F4BEC0D701EC93AA
:102AB00011963C93119712966C93129713967C93F0
:102AC000E4E0F0E0EE0EFF1EF6013196D60111961D
:102AD0000C911197112707FD109563CF0115110572
:102AE000C1F0903208F4A0C007FD9EC0003211056D
:102AF00081F00C30110569F00A30110551F00D30EC
:102B0000110539F00930110521F00B30110509F0DC
:102B10008BC0CE010196E81AF90AF594E794F59472
:102B2000E7940894E11CF11CB2E0EB16F10499F073
:102B3000E3E0EE16F1042CF4E114F10409F474C09E
:102B400062C0F3E0EF16F104E1F024E0E216F104D4
:102B500009F059C02FC0403030E0530730E0630720
:102B600031E0730708F060C089819A81AB81BC8134
:102B7000B82FAA2799278827482B592B6A2B7B2BFC
:102B800042C0403080E0580781E0680780E0780765
:102B900008F04AC00D811E812F81388598011127C8
:102BA000002789819A81AB81BC81B82FAA279927F8
:102BB000882721C04F3F51056105710509F0A0F537
:102BC0000D811E812F813885980111270027898169
:102BD0009A81AB81BC81B82FAA2799278827082B17
:102BE000192B2A2B3B2B89859A85AB85BC85BA2F5F
:102BF000A92F982F8827082B192B2A2B3B2B402BEA
:102C0000512B622B732BAB89BC89109781F0CB01C0
:102C1000BA010E947C14DC01CB01EB89FC89808322
:102C20009183A283B38303C080E090E002C081E07F
:102C300090E06496CDBFDEBFDF91CF911F910F91E1
:102C4000FF90EF90DF90CF90BF90AF909F908F90CC
:102C50007F906F905F904F903F902F9008950F93CB
:102C60001F93CF93DF93CDB7DEB72797CDBFDEBFDE
:102C7000FC0180819181A281B3818C839D83AE838D
:102C8000BF83AE014C5F5F4F20E0E4E3F3E31AE063
:102C90000EE2DA018C9130E0612F0E945F50A1E0DA
:102CA000B0E0AC0FBD1FA30FB11D905D9C933F5FC3
:102CB000882391F7632FDA011D92AD01CF010BC07C
:102CC0003150A1E0B0E0AC0FBD1FA30FB11D7C914E
:102CD000DC017D93CD01332399F7DF01A60FB11DF0
:102CE000FD0101932F5F2430A1F61C9284E393E34E
:102CF0002796CDBFDEBFDF91CF911F910F91089531
:102D000080E090E008950E94CF5008950F931F93A4
:102D1000CF93DF930F920F92CDB7DEB7AC0149830B
:102D20005A830E94CF508C0149815A81009721F02B
:102D300060E070E00E94A354C8010F900F90DF91F3
:102D4000CF911F910F9108950E94FE5108950E9406
:102D5000655108950E94885408950E94A3540895CF
:102D60000E9491540895FC0101900020E9F73197E9
:102D7000E81BF90BCF0108950E94095508950E94A0
:102D8000FB5408950E94D35408950E94DC54089582
:102D90000E9453540895EF92FF920F931F93CF9385
:102DA000DF937C01EB01CB0101960E94CF508C0197
:102DB000009739F0B701AE010E940955C00FD11F2D
:102DC0001882C801DF91CF911F910F91FF90EF9072
:102DD00008950E94BD5408950E947B5408950E9456
:102DE000DE5208950E94C85408950E94185508950F
:102DF0000E94AA5408950E94235508950E94765473
:102E000008950E94E3540895CF92DF92EF92FF92CB
:102E10000F931F93CF93DF937C01D62EC72EDC0137
:102E20000D900020E9F78D0101501040081B190B8F
:102E3000E62FF72FEF0109900020E9F72197CE1B2D
:102E4000DF0B0DC0C7016D2D7C2DAE010E94E35438
:102E5000009751F00894E11CF11C015010400C1730
:102E60001D0780F7EE24FF24C701DF91CF911F914A
:102E70000F91FF90EF90DF90CF900895CF93DF9365
:102E8000CDB7DEB79E01245F3F4F8E819F8168855D
:102E900079854A855B850E94BF55DF91CF91089562
:102EA0000E94BF550895EF92FF920F931F93CF9307
:102EB000DF93CDB7DEB7C05AD040CDBFDEBFC65519
:102EC000DF4FE880CA5AD040C555DF4FF880CB5A53
:102ED000D0409E0124553F4FCE01019660EA70E03C
:102EE000A7010E94BF558C0197FD05C07E01089483
:102EF000E11CF11C04C087010AC00E942B46F701A7
:102F000081917F018823C9F709C00E942B46F801EF
:102F100081918F018823C9F70FEF1FEFC801C056B9
:102F2000DF4FCDBFDEBFDF91CF911F910F91FF909B
:102F3000EF9008958F929F92AF92BF92CF92DF92BF
:102F4000EF92FF920F931F93CF93DF938C01009723
:102F5000B9F1DC011C968D919C911D970E94A716DA
:102F6000D8011296ED91FC911397E080F18022E058
:102F7000C22ED12CC00ED11EA12C31E0B32E812C3B
:102F800042E0942E17C0C281D381A081B1811296F4
:102F9000CD93DC931397A883B983A082B1828282F8
:102FA0009382CF0106970E94A716F7019081818135
:102FB000E92EF82EEC15FD0531F7C8010E94A71681
:102FC000DF91CF911F910F91FF90EF90DF90CF9005
:102FD000BF90AF909F908F900895CF92DF92EF9225
:102FE000FF920F931F93CF93DF93EC016B017A0154
:102FF00089018AE090E00E948616FC010097C9F0E2
:10300000C082D182E282F382048315839C012A5F0D
:103010003F4FAC81BD812C833D83CE0102968683D8
:103020009783A087B1872D933C93119780E090E020
:1030300002C08DEF9FEFDF91CF911F910F91FF9015
:10304000EF90DF90CF90089520E030E00E94ED17E0
:103050000895FC0162AB73AB44AB55AB0895FC0122
:10306000808191810895FC01848995898870907090
:103070000895FC0180A991A90895CF92DF92EF9263
:10308000FF920F931F93CF93DF93CDB7DEB7CC841E
:10309000DD848E01005F1F4F80E590E00E94831663
:1030A0007C010097F1F060E570E04E855F85980146
:1030B0000E945017AC0197FF04C0C7010E94A716D9
:1030C00010C0D6011896ED91FC9119971A968D9122
:1030D0009C911B97B70119958C01C7010E94A716F7
:1030E00002C00DEF1FEFC801DF91CF911F910F912B
:1030F000FF90EF90DF90CF9008954F925F926F9284
:103100007F928F929F92AF92BF92CF92DF92EF9277
:10311000FF920F931F93CF93DF93CDB7DEB76497E2
:10312000CDBFDEBF7C01DC0112960D911C9113977F
:1031300052E0A52EB12CA80EB91E6E010894C11C38
:10314000D11C64E1862E912C71E0672E70E2772EFF
:10315000E7E04E2EE0E25E2E55C0D8011697ED91C5
:10316000FC9111972081318114968D919C91159736
:10317000009711F480E090E2EDB7FEB73A97EDBF0B
:10318000FEBF3196ADB7BEB71196CD92DC921297C5
:1031900082829382648275822683378380879187B7
:1031A0000E943E17F80136970190F081E02D84814E
:1031B0009581EDB7FEB73A96EDBFFEBF009711F4CB
:1031C00080E090E22DB73EB7285030402DBF3EBF83
:1031D000EDB7FEB73196ADB7BEB71196ED92FC9242
:1031E000129742825382C482D582868397830E943B
:1031F0003D18F801008111812DB73EB7285F3F4F80
:103200002DBF3EBF0A151B0509F0A7CF6496CDBFA1
:10321000DEBFDF91CF911F910F91FF90EF90DF9074
:10322000CF90BF90AF909F908F907F906F905F9066
:103230004F900895EF92FF920F931F93CF93DF93D8
:103240008C01EB01DC0154968C91549783FF21C0D3
:1032500077FD03C082E190E202C085E190E2EDB724
:10326000FEB73897EDBFFEBF3196ADB7BEB711962A
:103270000D931C93129729E130E2228333838483D8
:103280009583C683D7830E943D18EDB7FEB7389665
:103290002CC077FD05C0A2E1EA2EA0E2FA2E04C000
:1032A000F5E1EF2EF0E2FF2ECE010E944C1F2DB76C
:1032B0003EB72A5030402DBF3EBFEDB7FEB7319626
:1032C000ADB7BEB711960D931C93129721E230E271
:1032D00022833383E482F582C683D78380879187F4
:1032E0000E943D18EDB7FEB73A96EDBFFEBFDF91E5
:1032F000CF911F910F91FF90EF9008952F923F92E1
:103300004F925F926F927F928F929F92AF92BF92F5
:10331000CF92DF92EF92FF920F931F93CF93DF93A1
:10332000CDB7DEB7C455D040CDBFDEBF6C011901AB
:10333000DC0154968C91549783FD27C0EDB7FEB7FE
:103340003897EDBFFEBF3196ADB7BEB71196CD929F
:10335000DC92129782E390E2828393836483758385
:103360002683378364964FAF649765965FAF659702
:103370000E943D18EDB7FEB73896EDBFFEBF6596CB
:103380005FAD659764964FAD64973A01AA24BB245C
:103390002E010894411C511C9E012F5A3F4F6396E9
:1033A0002EAF3FAF6397BAC0D60154968C91549715
:1033B00083FD21C0EDB7FEB73897EDBFFEBF319654
:1033C000ADB7BEB711964D925C92129720E530E0F2
:1033D000228333838AE490E284839583A682B78232
:1033E0000E943E174201880E991EADB7BEB71896CF
:1033F000ADBFBEBF01C04201740100E010E0C801D2
:103400008A0D9B1D821593056CF5EDB7FEB73897B5
:10341000EDBFFEBFADB7BEB71196E182F2826396F3
:103420008EAD9FAD63978E199F0912968D939C93D5
:10343000139721E530E214962D933C931597F301F1
:10344000E00FF11F8081992787FD909516968D9347
:103450009C9317970E943E178DB79EB708968DBF15
:103460009EBF05C0C7016EE270E20E94C516A3E0D0
:10347000B0E0EA0EFB1E0F5F1F4F0031110509F08F
:10348000BECFD401D096F601848983FD1AC020E016
:1034900030E0C9018A0D9B1D821593056CF4F30180
:1034A000E20FF31F4081CD010196403214F04C939E
:1034B00002C0FEE2FC93DC012F5F3F4F203131055B
:1034C00041F71C92D60154968C91549783FF03C008
:1034D00080E090E202C08EE290E2EDB7FEB738974E
:1034E000EDBFFEBF3196ADB7BEB71196CD92DC925F
:1034F000129727E530E222833383848395834682C3
:1035000057820E943D1880E190E0A80EB91E680E17
:10351000791EADB7BEB71896ADBFBEBFA214B30437
:103520000CF442CFCC5ADF4FCDBFDEBFDF91CF913D
:103530001F910F91FF90EF90DF90CF90BF90AF90D1
:103540009F908F907F906F905F904F903F902F90C3
:1035500008952F923F924F925F926F927F928F9237
:103560009F92AF92BF92CF92DF92EF92FF920F9312
:103570001F93CF93DF9300D0CDB7DEB78A839B83B1
:10358000DC0152968D919C9153970097D9F15096FA
:103590008D919C9151978F3491052CF052961D92EC
:1035A0001C92539734C26E3679F0623719F06C353D
:1035B000F9F415C0AA81BB811C96ED91FC911D9771
:1035C000E80FF91F8DE009C0AA81BB811C96ED911F
:1035D000FC911D97E80FF91F8AE0808309C0AA813A
:1035E000BB811C96ED91FC911D97E80FF91F60833C
:1035F000EA81FB81808991890196808B918B128A67
:10360000138A05C26A3009F43FC06B3024F4683075
:1036100009F0B6C113C06D30B9F16C3509F0B0C115
:10362000AA81BB8154968C91549782FF07C081E098
:1036300090E052968D939C935397E9C1EA81FB8168
:1036400080899189009709F4E2C1848981FD14C0C1
:1036500000D00F92ADB7BEB71196ED93FC931297C1
:103660008EE590E213968D939C9314970E943D18DB
:103670000F900F900F900F90EA81FB8180899189C4
:103680000197808B918BC3C1AA81BB811C96ED9160
:10369000FC911D9750968D919C915197E80FF91FC1
:1036A000108254968C91549781FD10C000D00F92D7
:1036B000EDB7FEB7A183B28382E690E28383948361
:1036C0000E943D180F900F900F900F90AA81BB8120
:1036D0001C968D919C911D9756961D921C92579702
:1036E00020E030E258962D933C9359975A962D93AB
:1036F0003C935B9719C0EA81FB8186899789FC011D
:103700003C96EE0FFF1F4A815B81E40FF51F20837B
:1037100031830196DA0156968D939C9357978C309E
:10372000910549F080E090E065E670E20E94FE16A7
:103730009C01009701F7EA81FB81A08CB18C428C3F
:10374000538CC280D380662477248824992492E005
:10375000292E312C2E0E3F1E48C0860106501040E7
:10376000D801ED91FC9180819181B5010E94C21632
:10377000009751F4F80184819581009729F0B201F6
:103780000E94C2160097D1F18AEFE82E8FEFF82E33
:10379000EC0CFD1CD701ED91FC9180819181B5016C
:1037A0000E94C216009729F4F70184819581009741
:1037B00029F1D701ED91FC91E080F180C5010E94D3
:1037C000B316AC01C701B5010E94BF16009721F4E2
:1037D0008114910419F405C0840103C0B1E06B2E7B
:1037E000712CF601C080D1804801C214D30409F0C5
:1037F000B4CF6114710409F055C08401011511059D
:1038000009F450C0D80112968D919C911397EA81CA
:10381000FB8180839183828D938D009759F114965B
:103820006D917C9115976115710521F10E94C21669
:10383000009701F5D80114968D919C911597EA8116
:10384000FB8180AB91AB808D918D828F938F668948
:10385000778961507040668B778BED91FC91119761
:103860004A815B81465E5F4F0280F381E02D8A8151
:103870009B8116C0AA81BB81D0961D921C92D197C4
:10388000D801ED91FC91AA81BB8156966D917C91F6
:103890005797AD01485E5F4F0280F381E02DCD0167
:1038A000199544C0AA81BB81D296ED91FC91D39722
:1038B000309741F0D4968D919C91D5978D939C93A0
:1038C0001197E3CFEA81FB81808D918D0E94B31621
:1038D000009761F1AA81BB8154968C91549783FF24
:1038E00006C0CD0169EE7FEF0E941A191FC000D0FB
:1038F00000D0EDB7FEB731964A815B81ADB7BEB758
:1039000011964D935C93129787E690E2828393839E
:10391000DA0158968D919C915997848395830E94E2
:103920003D18EDB7FEB73696EDBFFEBFAA81BB814D
:1039300050961D921C92519754968C91549780FDED
:1039400066C000D000D0EDB7FEB73196AD01ADB77F
:10395000BEB711964D935C9312978EE790E28283E7
:103960009383DA0116968D919C91179784839583A2
:103970000E943D18EDB7FEB73696EDBFFEBF47C0BB
:10398000AA81BB8150968D919C9151978F3491055E
:10399000F4F5862F80528F35D0F554968C9154973C
:1039A00081FD1FC000D000D0EDB7FEB73196AD014C
:1039B000ADB7BEB711964D935C93129782E890E233
:1039C00082839383862F992787FD9095848395839F
:1039D00069830E943D188DB79EB706968DBF9EBF26
:1039E0006981AA81BB811C96ED91FC911D9750962F
:1039F0008D919C915197E80FF91F608350968D919E
:103A00009C915197019650968D939C935197239634
:103A1000CDBFDEBFDF91CF911F910F91FF90EF904F
:103A2000DF90CF90BF90AF909F908F907F906F90DE
:103A30005F904F903F902F900895CF92DF92EF923A
:103A4000FF920F931F93CF93DF936C017A018B0149
:103A5000C0E0D0E007C0F80161918F01C6010E946B
:103A6000A91A2196CE15DF05B4F3C701DF91CF91D6
:103A70001F910F91FF90EF90DF90CF900895AF923C
:103A8000BF92CF92DF92EF92FF920F931F93CF934B
:103A9000DF93EC016B015A01F22EE32E61157105E3
:103AA00009F45DC023FD5BC086E390E00E948316AD
:103AB0008C01009709F455C060E070E046E350E0E7
:103AC0000E94AD16209711F4C5E8D0E2D8011696F1
:103AD000CD93DC93179780E590E01E968D939C9391
:103AE0001F970E948316F80184879587009721F419
:103AF000C8010E949A1733C04685578560E070E080
:103B00000E94AD16F801F48AE58AC086D186A286A5
:103B1000B386C80102968283938384839583F0FCE5
:103B200020C000D000D0EDB7FEB73196ADB7BEB71C
:103B300011960D931C9312978EE790E282839383E4
:103B4000D80116968D919C911797848395830E9436
:103B50003D18EDB7FEB73696EDBFFEBF02C000E0E0
:103B600010E0C801DF91CF911F910F91FF90EF906E
:103B7000DF90CF90BF90AF9008952F923F924F92D9
:103B80005F926F927F928F929F92AF92BF92CF92ED
:103B9000DF92EF92FF920F931F93CF93DF930F92D9
:103BA0000F92CDB7DEB74C0181E090E069837A8354
:103BB0000E9486168C0169817A81009709F44EC0B3
:103BC0007B01CC24DD24240108944108510842C023
:103BD00051E0A52EB12CC414D50414F0AA24BB24A2
:103BE000C8010E94B3161C013701F7018081918141
:103BF0000E94B316B5016F5F7F4F620D731D680F92
:103C0000791FC8010E94A4161C01009731F4C80155
:103C10000E94A71600E010E021C00E94B31622E027
:103C200030E0E20EF31EF30160817181820D931D7D
:103C30000E94C516A114B10449F0C1010E94B31637
:103C4000820D931D65E670E20E94C5160894C11CA2
:103C5000D11C8101C814D9040CF4BACFC8010F904B
:103C60000F90DF91CF911F910F91FF90EF90DF9018
:103C7000CF90BF90AF909F908F907F906F905F900C
:103C80004F903F902F9008953F924F925F926F9286
:103C90007F928F929F92AF92BF92CF92DF92EF92DC
:103CA000FF920F931F93CF93DF93CDB7DEB7C45529
:103CB000D040CDBFDEBF4A0100D000D0EDB7FEB787
:103CC000319623EA30E2ADB7BEB711962D933C93FF
:103CD0001297828393834483558364966FAF64976E
:103CE00065967FAF65970E94531764966FAD649792
:103CF000A62E65967FAD6597B72EEDB7FEB73696C3
:103D0000EDBFFEBFCC24DD24CE018F5A9F4F6396BA
:103D10008EAF9FAF63972E010894411C511C6EE239
:103D2000362EA0C0ADB7BEB71897ADBFBEBFEDB7BA
:103D3000FEB7319611964D925C92129780E590E015
:103D400082839383ABEBB0E2A483B583C682D78230
:103D50000E943E173201680E791EEDB7FEB7389605
:103D6000EDBFFEBF730100E010E0C8018C0D9D1D8A
:103D7000881599056CF58DB79EB708978DBF9EBFC6
:103D8000ADB7BEB71196EDB7FEB7E182F28263968A
:103D90008EAD9FAD63978E199F0912968D939C935C
:103DA000139782EC90E214968D939C931597F501EE
:103DB000E00FF11F808116968C93169717961C9230
:103DC0000E943E17ADB7BEB71896ADBFBEBF05C0C7
:103DD000C70168EC70E20E94C516E3E0F0E0EE0E69
:103DE000FF1E0F5F1F4F0031110509F0BECF830189
:103DF000005D1F4FC8016CEC70E20E94C51640E0E8
:103E000050E0CA018C0D9D1D8815990574F4F501CB
:103E1000E40FF51F2081C801019620321CF0D80163
:103E20002C9302C0F80130828C014F5F5F4F40310C
:103E3000510539F7D8011C9200D00F928FEC90E217
:103E4000EDB7FEB781839283438254820E94531759
:103E5000A0E1B0E0CA0EDB1EAA0EBB1E0F900F90B1
:103E60000F900F90C814D9040CF45CCFCC5ADF4FDC
:103E7000CDBFDEBFDF91CF911F910F91FF90EF90EB
:103E8000DF90CF90BF90AF909F908F907F906F907A
:103E90005F904F903F900895FC0197FF0BC076967E
:103EA000E631F10550F4EE0FFF1FE25FFD4C80811B
:103EB0009181089587ED90E208958FED90E2089545
:103EC00086E090E00E9486168093483390934933B1
:103ED000009719F48DEF9FEF089580E090E008952A
:103EE000CF93DF930097B1F1A0914833B09149335C
:103EF00014962C91149720FF07C0FC01268137816E
:103F000024602683378326C02D913C911197F901B7
:103F1000C0E0D0E01AC0E817F90731F050814181C4
:103F2000EF01E52FF42F11C0209739F4F90120811A
:103F300031812D933C93119705C0FC012081318183
:103F4000288339830E94A71605C0309721F78EEF8A
:103F50009FEF02C080E090E0DF91CF910895FC01D7
:103F6000A0914833B091493312968D919C9113974B
:103F70008087918762877387868197818E7F86830A
:103F800097830895AF92BF92CF92DF92EF92FF9204
:103F90000F931F93CF93DF935C018B01EA016901BB
:103FA000209769F18CE090E00E9486167C010097D2
:103FB00041F1FC01C283D383C482D582011511056E
:103FC00029F086819781826086839783A091483308
:103FD000B0914933ED91FC911197309729F4ED920E
:103FE000FC92119707C0FC01808191810097D9F75D
:103FF000E082F182C701B5010E94AF1F02C0EE242A
:10400000FF24C701DF91CF911F910F91FF90EF9097
:10401000DF90CF90BF90AF900895E0914833F0913A
:104020004933828193810895E0914833F091493377
:10403000309731F022813381280F391F2283338357
:1040400008954115510519F086179707D1F06817A3
:10405000790750F0681B790B81E090E064177507D1
:1040600090F480E090E0089580959095860F971FDA
:1040700021E030E08417950710F420E030E0C9011A
:10408000089580E090E008950F931F93CF93DF93FE
:10409000E0914833F0914933848195818160848334
:1040A0009583C081D18129C00E811F81C80185708F
:1040B00090700097F9F4E0914833F09149336281B0
:1040C00073814A855B85888599850E9421200097A8
:1040D00089F001600E831F836C817D81EA81FB8101
:1040E000CE0119958E8181FF05C06A857B85CE0141
:1040F0000E94AF1F0990D881C02D2097A9F6E091AA
:104100004833F0914933848195818E7F84839583F0
:104110000190F081E02D00E010E024C0868182FF54
:104120001CC00115110561F4C0914833D091493389
:10413000A881B9818D919C9111978883998305C03D
:1041400080819181D8018D939C93D081C181CF01D1
:104150000E94A716ED2FFC2F05C0908181818F0151
:10416000E92FF82F3097D1F6DF91CF911F910F9162
:104170000895EF92FF920F931F93CF93DF938C01DB
:10418000C0914833D0914933EA80FB806A817B81BA
:10419000C701A8010E9421200097C1F3DF91CF91B0
:1041A0001F910F91FF90EF9008956817790728F4F9
:1041B00080959095860F971F08959B01281B390BBA
:1041C000C9010895CF93DF93DC01FB0180839183C4
:1041D000EC0120E030E026C0863271F41C922417F6
:1041E0003507FCF4F901EE0FFF1FEE0FFF1FE60F7E
:1041F000F71FC083D18315C08D3399F4F901EE0FF9
:10420000FF1FEE0FFF1FE60FF71F808191810097C0
:1042100041F01C922417350724F4C283D3832F5F07
:104220003F4F119689918823B9F6C901DF91CF914B
:104230000895AF92BF92CF92DF92EF92FF920F93C9
:104240001F93CF93DF935C016A01EB01EE24FF24FF
:1042500000E010E00FC0688179816115710569F097
:10426000C5010E94C216009711F4EA80FB800F5F1F
:104270001F4F24960C151D0574F3C701DF91CF91D4
:104280001F910F91FF90EF90DF90CF90BF90AF9074
:1042900008958DE290E061E070E00E9445468EE274
:1042A00090E062E070E00E9445468EE290E00E945D
:1042B000AD4689E290E062E070E00E94454689E206
:1042C00090E00E94984684EF91E00E941D4689E2AA
:1042D00090E00E94AD4684EF91E00E941D4680E090
:1042E00090E0089589E290E062E070E00E94454627
:1042F00089E290E00E94984680E090E008952DB712
:104300003EB72A5030402DBF3EBFEDB7FEB73196C5
:10431000ADB7BEB711968D939C93129785E192E24B
:104320008283938381E090E08483958383E090E0AF
:104330008683978382E090E0808791870E943D1872
:104340002DB73EB7265F3F4F2DBF3EBF08952DB717
:104350003EB7285030402DBF3EBFEDB7FEB7319677
:10436000ADB7BEB711968D939C9312978BE292E2F4
:104370008283938364837583468357830E943D18A9
:104380002DB73EB7285F3F4F2DBF3EBF08950F9317
:104390001F93CF93DF938C01EB010E94B316482F3C
:1043A00088A3CE01B80150E00E94AA1681E090E0F7
:1043B000DF91CF911F910F910895EF92FF920F938C
:1043C0001F93CF93DF93CDB7DEB7A197CDBFDEBFED
:1043D0008C01623071057CF0DA0112968D919C910E
:1043E0001397BE016F5F7F4F0E94C7210097F1F1C5
:1043F000CE01019602C080E090E06AE670E3A80179
:104400000E94F50B7C01C8010E943318009749F106
:10441000F7FE05C081E592E225E532E204C08CE4B6
:1044200092E22FE432E2EDB7FEB73A97EDBFFEBF5E
:104430003196ADB7BEB711960D931C93129746E512
:1044400052E24283538384839583E682F7822087F6
:1044500031870E943D18EDB7FEB73A96EDBFFEBF1B
:1044600019C0C801B7010E941A1914C000D00F92D8
:10447000ADB7BEB711960D931C93129780E692E2EA
:1044800013968D939C9314970E943D180F900F9054
:104490000F900F90A196CDBFDEBFDF91CF911F91FE
:1044A0000F91FF90EF900895EF92FF920F931F935B
:1044B000CF93DF930F920F92CDB7DEB77C018B01C4
:1044C000BE016F5F7F4F40E050E00E94EF16DC01BD
:1044D000CB01F80180839183A283B38301E010E0D4
:1044E00020E030E089819A818E159F0519F400E063
:1044F00010E09801B801C9010F900F90DF91CF91A2
:104500001F910F91FF90EF9008950F931F93CF93FA
:10451000DF9300D00F92CDB7DEB78C01623071050A
:10452000CCF0FA0182819381BE016F5F7F4F0E94C0
:104530005422DC01CB010097A105B10559F0698136
:104540007A818B819C810E945614BC01C8010E9413
:104550001A1910C000D00F92EDB7FEB70183128375
:1045600084E792E2838394830E943D180F900F901A
:104570000F900F902496CDBFDEBFDF91CF911F919A
:104580000F910895EF92FF920F931F93CF93DF93B4
:104590000F920F92CDB7DEB77C018B01BE016F5F2A
:1045A0007F4F40E050E00E94EF16DC01CB01F801A4
:1045B0008083918381E090E029813A812E153F0527
:1045C00011F480E090E00F900F90DF91CF911F9158
:1045D0000F91FF90EF900895EF92FF920F931F932A
:1045E000CF93DF930F920F92CDB7DEB78C017B0193
:1045F000BE016F5F7F4F40E050E00E94EF16AB01BD
:10460000BC0189819A818017910741F057FD06C04E
:10461000F7014083518381E090E002C080E090E0A8
:104620000F900F90DF91CF911F910F91FF90EF901E
:104630000895EF92FF920F931F93CF93DF9300D0D3
:104640000F92CDB7DEB78C0162307105B4F1DA019B
:1046500012968D919C911397BE016F5F7F4F0E94C0
:104660005422DC01CB010097A105B10531F169812C
:104670007A818B819C810E9438147C0100D000D00B
:10468000EDB7FEB73196ADB7BEB711960D931C933B
:1046900012978CE992E28283938389819A81848341
:1046A00095830E943D18EDB7FEB73696EDBFFEBF6D
:1046B000C801B7010E941A1914C000D00F92ADB7FB
:1046C000BEB711960D931C93129788EA92E2139647
:1046D0008D939C9314970E943D180F900F900F900C
:1046E0000F902496CDBFDEBFDF91CF911F910F9128
:1046F000FF90EF9008950F931F93CF93DF930F9246
:104700000F92CDB7DEB78C01623071059CF0FA01D3
:1047100082819381BE016F5F7F4F0E94C22200970A
:1047200049F089819A810E942414BC01C8010E9429
:104730001A1910C000D00F92EDB7FEB70183128393
:1047400085EC92E2838394830E943D180F900F9032
:104750000F900F900F900F90DF91CF911F910F91BD
:1047600008950F931F93CF93DF930F92CDB7DEB7CA
:104770008C01CE0101960E94710ABC01C8010E9401
:104780001A1900D000D0EDB7FEB73196ADB7BEB75D
:1047900011960D931C9312978CED92E28283938372
:1047A0008981848315820E943D188DB79EB7069635
:1047B0008DBF9EBF0F90DF91CF911F910F910895F4
:1047C000CF92DF92EF92FF920F931F93CF93DF93DD
:1047D000CDB7DEB7A497CDBFDEBF7C0125E1C22EE9
:1047E000D12CCC0EDD1ECE010196B60140E150E089
:1047F0009E012B5F3F4F00E110E00E947F0BBC0148
:10480000C7010E941A1949815A816B817C818DB739
:104810009EB70C978DBF9EBFEDB7FEB73196ADB773
:10482000BEB71196ED92FC92129782EF92E28283CC
:104830009383862F90E084839583BB27A72F962FA1
:10484000852F907086839783507040875187C286EA
:10485000D3860E943D188DB79EB70C968DBF9EBF24
:10486000CE0105960E94B316009719F0CE01059669
:1048700002C08AEE92E200D000D0EDB7FEB73196CA
:10488000ADB7BEB71196ED92FC92129721E133E2DB
:1048900022833383848395830E943D188DB79EB70E
:1048A00006968DBF9EBFA496CDBFDEBFDF91CF9190
:1048B0001F910F91FF90EF90DF90CF900895AF92EE
:1048C000BF92CF92DF92EF92FF920F931F93CF93FD
:1048D000DF9300D00F92CDB7DEB75C018B017A0178
:1048E000CE01019660E070E040E050E020E030E072
:1048F0000E946C0CC80101978530910508F070C0CA
:104900000130110509F481C0D70112968D919C9157
:10491000139762E273E20E94C216009709F060C02A
:104920000230110509F471C0F70184819581BE013F
:104930006F5F7F4F0E94AA14009709F451C00330A3
:10494000110509F462C0D70116968D919C911797B5
:1049500060E070E04AE050E00E94EF16DC01CB011D
:104960006C010530110521F4F7010085118502C0A5
:1049700000E010E080E0BE016F5F7F4FA60198016C
:104980000E94B913BC01C5010E941A19CE010196FB
:104990000E942F160115110511F405E512E22DB73D
:1049A0003EB72A5030402DBF3EBFEDB7FEB731961F
:1049B000ADB7BEB71196AD92BC9212972CE233E21E
:1049C0002283338384839583C682D78200871187AD
:1049D0000E943D18EDB7FEB73A96EDBFFEBF1AC074
:1049E00000D00F92ADB7BEB71196AD92BC921297A0
:1049F00084E493E213968D939C9314970E943D1840
:104A00000F900F900F900F9005C080E9C82E8FE196
:104A1000D82EAECF2496CDBFDEBFDF91CF911F91B0
:104A20000F91FF90EF90DF90CF90BF90AF900895DF
:104A30000F931F93CF93DF93CDB7DEB76097CDBFB2
:104A4000DEBF8C01CE010D96BE01675F7F4FAE01C8
:104A50004B5F5F4F9E012F5F3F4F0E946C0C97FD95
:104A600003C02CE432E202C021E532E24DB75EB76A
:104A7000485050404DBF5EBFEDB7FEB73196ADB761
:104A8000BEB711960D931C93129748E853E24283E8
:104A9000538324833583868397830E943D184DB7C3
:104AA0005EB7485F5F4F4DBF5EBFCE010D960E945F
:104AB0002F1600D000D0EDB7FEB73196ADB7BEB718
:104AC00011960D931C93129720E933E222833383CE
:104AD000848395830E943D184DB75EB74A5F5F4F50
:104AE0004DBF5EBFCE0109960E942F1600D000D0A8
:104AF000EDB7FEB73196ADB7BEB711960D931C93C7
:104B0000129727E933E222833383848395830E94BB
:104B10003D184DB75EB74A5F5F4F4DBF5EBFCE01D8
:104B200005960E942F1600D000D0EDB7FEB7319643
:104B3000ADB7BEB711960D931C93129720EA33E2DE
:104B400022833383848395830E943D184DB75EB7DB
:104B50004A5F5F4F4DBF5EBFCE0101960E942F1688
:104B600000D000D0EDB7FEB73196ADB7BEB7119605
:104B70000D931C93129727EA33E2228333838483B5
:104B800095830E943D184DB75EB74A5F5F4F4DBF9A
:104B90005EBF6096CDBFDEBFDF91CF911F910F91B9
:104BA00008950F931F93CF93DF9300D000D0CDB71C
:104BB000DEB78C0162307105A4F1DA0112968D9195
:104BC0009C911397BE016F5F7F4F0E94C222009796
:104BD00041F189819A81BE016D5F7F4F0E94AB10C8
:104BE000BC01C8010E941A19CE0103960E942F161B
:104BF00000D000D0EDB7FEB73196ADB7BEB7119675
:104C00000D931C93129721EB33E222833383848329
:104C100095830E943D18EDB7FEB73696EDBFFEBFF7
:104C200014C000D00F92ADB7BEB711960D931C9370
:104C300012978BEB93E213968D939C9314970E949B
:104C40003D180F900F900F900F902696CDBFDEBFAE
:104C5000DF91CF911F910F9108952F923F924F9224
:104C60005F926F927F928F929F92AF92BF92CF92FC
:104C7000DF92EF92FF920F931F93CF93DF93CDB705
:104C8000DEB72897CDBFDEBF4C017B018A016430BF
:104C900071050CF4A6C0DA0112968D919C911397C0
:104CA000BE016D5F7F4F0E94C222009709F499C038
:104CB00025E0A22EB12CAC0EBD1EF8018481958199
:104CC000B5010E94AA14009709F48BC0D80116966A
:104CD0008D919C911797BE016F5F7F4F0E94EC22D0
:104CE000009709F47EC0B801685F7F4FC701049741
:104CF0000E94BD1D6C01009709F46CC00E94B316A0
:104D00003C01C5010E942F16EDB7FEB73A97EDBFE3
:104D1000FEBF3196ADB7BEB711968D929C92129799
:104D20002AED33E2228333836482758286839783FC
:104D300089819A81808791870E943D18EDB7FEB7DF
:104D40003A96EDBFFEBFEE24FF24250196EF292EF3
:104D500093E2392E36C05301AE18BF08B6016E0D6E
:104D60007F1D09811A818B819C81A50192010E947E
:104D700031108C0197FF04C0C6010E9465512CC000
:104D80002DB73EB7285030402DBF3EBFEDB7FEB720
:104D90003196ADB7BEB711968D929C921297228232
:104DA000338284839583C501801B910B868397830F
:104DB0000E943D18E00EF11EEDB7FEB73896EDBF2C
:104DC000FEBFE614F7043CF2C6010E94655100E004
:104DD00010E002C00DEF1FEFC401B8010E941A19C4
:104DE00014C000D00F92ADB7BEB711968D929C92B1
:104DF00012978BE094E213968D939C9314970E94E4
:104E00003D180F900F900F900F902896CDBFDEBFEA
:104E1000DF91CF911F910F91FF90EF90DF90CF9096
:104E2000BF90AF909F908F907F906F905F904F90CA
:104E30003F902F9008954F925F926F927F928F9242
:104E40009F92AF92BF92CF92DF92EF92FF920F9319
:104E50001F93CF93DF930F920F92CDB7DEB74C0124
:104E60007B018A01633071050CF47CC0DA01129673
:104E70008D919C911397BE016F5F7F4F0E94C2225C
:104E8000009709F46FC0B8016C5F7F4FC7010297AC
:104E90000E94BD1D6C01009709F45DC00E94B3160D
:104EA0005C0100D000D0EDB7FEB73196ADB7BEB70C
:104EB00011968D929C9212978BE394E28283938356
:104EC000A482B5820E943D18EDB7FEB73696EDBFBD
:104ED000FEBFEE24FF2436EF432E33E2532E32C0C2
:104EE00035016E187F08B6016E0D7F1D89819A818C
:104EF000A3010E94CD0F8C0197FF04C0C6010E9440
:104F000065512BC08DB79EB708978DBF9EBFEDB77B
:104F1000FEB73196ADB7BEB711968D929C9212979F
:104F20004282538204831583C301801B910B8683C5
:104F300097830E943D18E00EF11EEDB7FEB738963C
:104F4000EDBFFEBFEA14FB045CF2C6010E9465518E
:104F500000E010E002C00DEF1FEFC401B8010E9495
:104F60001A1914C000D00F92ADB7BEB711968D922A
:104F70009C9212978EE494E213968D939C931497CF
:104F80000E943D180F900F900F900F900F900F9070
:104F9000DF91CF911F910F91FF90EF90DF90CF9015
:104FA000BF90AF909F908F907F906F905F904F9049
:104FB00008950F931F93CF93DF930F920F92CDB766
:104FC000DEB78C01623071059CF0FA018281938119
:104FD000BE016F5F7F4F0E94C222009749F0898116
:104FE0009A810E94BF0EBC01C8010E941A1910C00C
:104FF00000D00F92EDB7FEB70183128380E794E2F1
:10500000838394830E943D180F900F900F900F9010
:105010000F900F90DF91CF911F910F910895EF9214
:10502000FF920F931F93CF93DF93CDB7DEB72897EF
:10503000CDBFDEBF7C018A016430710564F1FA01E5
:1050400082819381BE016D5F7F4F0E94C2220097D3
:1050500011F1F80184819581BE016B5F7F4F0E9441
:10506000AA140097C1F0F80186819781BE016F5F95
:105070007F4F0E94EC22009771F049815A818B8109
:105080009C81BE016B5F7F4F0E94330EBC01C70144
:105090000E941A1910C000D00F92EDB7FEB7E1823E
:1050A000F28288E894E2838394830E943D180F90F3
:1050B0000F900F900F902896CDBFDEBFDF91CF915C
:1050C0001F910F91FF90EF900895CF92DF92EF9292
:1050D000FF920F931F93CF93DF9300D00F92CDB722
:1050E000DEB76C017B018A0181E090E089839A83BD
:1050F0006230710534F1FA0182819381BE016D5FE6
:105100007F4F0E94C2220097E1F0F2E0EF16F10417
:1051100051F0F80184819581BE016F5F7F4F0E943D
:10512000C222009771F069817A818B819C814DEB5D
:1051300058E296010E94F80DBC01C6010E941A199E
:1051400010C000D00F92EDB7FEB7C182D2828EEAB6
:1051500094E2838394830E943D180F900F900F90E8
:105160000F902496CDBFDEBFDF91CF911F910F919D
:10517000FF90EF90DF90CF9008950F931F93CF9300
:10518000DF938C01EB0100D000D0EDB7FEB7319674
:10519000ADB7BEB711968D939C93129781ED94E2B3
:1051A00082839383648375830E943D188DB79EB775
:1051B00006968DBF9EBFCE010E94750EEC0118169B
:1051C00019065CF467EA71E2A8010E94930DCE0112
:1051D00066EF78E2A8010E94AC0DC801BE010E94F2
:1051E0001A19DF91CF911F910F910895AF92BF923D
:1051F000CF92DF92EF92FF920F931F93CF93DF93A3
:10520000CDB7DEB7C054D040CDBFDEBF6C015B016F
:105210008A014115510519F085E592E202C085EF3A
:1052200094E22DB73EB72A5030402DBF3EBFEDB7B8
:10523000FEB73196ADB7BEB71196CD92DC921297FC
:1052400027E035E222833383A482B5820683178365
:10525000808791870E943D182DB73EB7265F3F4F4C
:105260002DBF3EBF15C0C501BE016F5F7F4FA701B7
:105270000E94170F9C0118161906ACF7081B190B92
:10528000C60165E275E2AE014F5F5F4F0E947E1975
:10529000101611064CF40134110518F080E490E06A
:1052A00001C0C8017C01DFCFC05CDF4FCDBFDEBFD6
:1052B000DF91CF911F910F91FF90EF90DF90CF90F2
:1052C000BF90AF900895EF92FF920F931F93CF93EB
:1052D000DF93CDB7DEB72897CDBFDEBF7C018A0153
:1052E0006430710564F1FA0182819381BE016D5FC2
:1052F0007F4F0E94C222009711F1F80184819581AD
:10530000BE016B5F7F4F0E94AA140097C1F0F801A5
:1053100086819781BE016F5F7F4F0E94EC220097CC
:1053200071F049815A818B819C81BE016B5F7F4FF7
:105330000E94C50DBC01C7010E941A1910C000D0FF
:105340000F92EDB7FEB7E182F28288E295E28383A5
:1053500094830E943D180F900F900F900F90289605
:10536000CDBFDEBFDF91CF911F910F91FF90EF90E6
:105370000895AF92BF92CF92DF92EF92FF920F9378
:105380001F93CF93DF930F920F92CDB7DEB76C01CF
:105390005B018A0119821A82623071050CF449C0DE
:1053A000FA01828193816BE475E20E94C216009734
:1053B000B1F0F8018281938162E575E20E94C21624
:1053C000009781F0F8018281938168E575E20E947F
:1053D000C216009771F552E0E52EF12C06C0EE24BE
:1053E000FF2403C041E0E42EF12CF2E0AF16B1043B
:1053F00051F0F80184819581BE016F5F7F4F0E945B
:10540000C2220097B1F069817A81C7010E943C0DE8
:105410008C0167EA71E2A6010E94930DC80166EF54
:1054200078E2A6010E94AC0DC601B8010E941A19CB
:1054300010C000D00F92EDB7FEB7C182D2828CE5CA
:1054400095E2838394830E943D180F900F900F90F4
:105450000F900F900F90DF91CF911F910F91FF90C0
:10546000EF90DF90CF90BF90AF9008950F931F9370
:10547000CF93DF930F920F92CDB7DEB78C016230DE
:1054800071059CF0FA0182819381BE016F5F7F4FAD
:105490000E94C222009749F089819A810E94AD0C36
:1054A000BC01C8010E941A1910C000D00F92EDB7BC
:1054B000FEB7018312838AE895E2838394830E9476
:1054C0003D180F900F900F900F900F900F90DF915D
:1054D000CF911F910F9108950F931F93CF93DF9357
:1054E0000F920F92CDB7DEB78C01CE0101960E94CC
:1054F000910C97FD03C02CE432E202C021E532E2B8
:105500004DB75EB74A5050404DBF5EBFEDB7FEB7D6
:105510003196ADB7BEB711960D931C93129743EA1F
:1055200055E242835383248335838683978389811D
:105530009A81808791870E943D184DB75EB7465F7C
:105540005F4F4DBF5EBF0F900F90DF91CF911F91C6
:105550000F9108950F931F93CF93DF930F920F92A4
:10556000CDB7DEB78C01623071059CF0FA01828103
:105570009381BE016F5F7F4F0E94C222009749F066
:1055800089819A810E94810CBC01C8010E941A196C
:1055900010C000D00F92EDB7FEB70183128388EBE5
:1055A00095E2838394830E943D180F900F900F9093
:1055B0000F900F900F90DF91CF911F910F91089551
:1055C000CF92DF92EF92FF920F931F93CF93DF93CF
:1055D000CDB7DEB76097CDBFDEBF6C017B018A011E
:1055E0008091043290910532A0910632B091073239
:1055F00089879A87AB87BC878D839E83AF83B88763
:1056000089839A83AB83BC83623071050CF446C0F6
:10561000FA0182819381BE01635F7F4F0E94AA14C9
:105620000097E1F1F2E0EF16F10431F1F801848125
:105630009581BE01675F7F4F0E94AA14009771F1A8
:10564000F3E0EF16F104C1F0F80186819781BE0105
:105650006B5F7F4F0E94AA14009701F1F4E0EF16F0
:10566000F10451F0F80180859185BE016F5F7F4F95
:105670000E94AA14009791F0CE010D96BE01675FBB
:105680007F4FAE014B5F5F4F9E012F5F3F4F0E94E8
:10569000630CBC01C6010E941A1910C000D00F9201
:1056A000EDB7FEB7C182D28280ED95E28383948309
:1056B0000E943D180F900F900F900F906096CDBFF5
:1056C000DEBFDF91CF911F910F91FF90EF90DF90A0
:1056D000CF900895EF92FF920F931F93CF93DF9394
:1056E000CDB7DEB7C155D040CDBFDEBF7C01CE0106
:1056F00082960E94F30C8C0197FD03C08CE492E229
:1057000002C081E592E22DB73EB7285030402DBF50
:105710003EBFEDB7FEB73196ADB7BEB71196ED926D
:10572000FC9212972FEF35E2228333838483958393
:10573000068317830E943D18EDB7FEB73896EDBF7C
:10574000FEBF0115110579F000D00F92ADB7BEB7BD
:105750001196ED92FC92129785E096E213968D9346
:105760009C931497C7C023964FAD2397CE01019603
:10577000BE016E5D7F4F50E00E94AA1623968FAD4A
:105780002397E1E0F0E0EC0FFD1FE80FF11D108220
:10579000882319F0CE01019602C08BEF95E2EDB798
:1057A000FEB77297EDBFFEBF3196ADB7BEB711968B
:1057B000ED92FC92129728E036E2228333838483B1
:1057C000958324968FAD24978683178225968FAD77
:1057D00025978087118626968FAD26978287138618
:1057E00027968FAD27978487158628968FAD2897A3
:1057F0008687178629968FAD2997808B118A0E94FC
:105800003D182B968EAD9FAD2B97EDB7FEB77296D8
:10581000EDBFFEBFFFEF80389F07C9F000D000D07A
:10582000EDB7FEB73196ADB7BEB71196ED92FC92CB
:1058300012972CE236E222833383848395830E947D
:105840003D18EDB7FEB73696EDBFFEBF14C000D0D1
:105850000F92ADB7BEB71196ED92FC92129785E309
:1058600096E213968D939C9314970E943D180F9087
:105870000F900F900F902D968EAD9FAD2D97BFEF8F
:1058800080389B07C9F000D000D0EDB7FEB7319645
:10589000ADB7BEB71196ED92FC9212972FE336E2A8
:1058A00022833383848395830E943D18EDB7FEB72E
:1058B0003696EDBFFEBF14C000D00F92ADB7BEB795
:1058C0001196ED92FC92129786E496E213968D93D0
:1058D0009C9314970E943D180F900F900F900F907B
:1058E00000D00F92EDB7FEB7E182F2828EE496E22D
:1058F000838394830E943D180F900F900F900F9018
:10590000CF5ADF4FCDBFDEBFDF91CF911F910F91F7
:10591000FF90EF9008950F931F93CF93DF9300D0E4
:1059200000D0CDB7DEB78C01CE0101960E94C60C27
:1059300097FD03C02CE432E202C021E532E24DB70C
:105940005EB7445150404DBF5EBFEDB7FEB73196D4
:10595000ADB7BEB711960D931C93129742E556E270
:105960004283538324833583868397838981808709
:1059700011868A81828713868B81848715868C8124
:10598000868717868D81808B118A8E81828B138A00
:105990000E943D184DB75EB74C5E5F4F4DBF5EBF76
:1059A0002696CDBFDEBFDF91CF911F910F91089555
:1059B0000F931F93CF93DF930F920F92CDB7DEB764
:1059C0008C016230710594F0FA0182819381BE01ED
:1059D0006F5F7F4F0E94C222009741F089810E9431
:1059E0004A13BC01C8010E941A1910C000D00F92BE
:1059F000EDB7FEB7018312838AE796E2838394832F
:105A00000E943D180F900F900F900F900F900F90E5
:105A1000DF91CF911F910F910895CF92DF92EF9276
:105A2000FF920F931F93CF93DF9300D000D0CDB799
:105A3000DEB76C017B018A0164307105ACF1FA01BB
:105A400082819381BE016B5F7F4F0E94C2220097CB
:105A500059F1F80184819581BE016D5F7F4F0E94ED
:105A6000C222009709F1F80186819781BE016F5F1C
:105A70007F4F0E94C2220097B9F0F4E0EF16F104C4
:105A800021F0F8012085318502C020E030E06B81F3
:105A90007C8149815A818D819E810E945A13BC016B
:105AA000C6010E941A191AC000D00F92EDB7FEB7B6
:105AB000C182D28289E996E2838394830E943D1851
:105AC000EDB7FEB7C182D28282EC96E283839483E3
:105AD0000E943D180F900F900F900F902696CDBF0B
:105AE000DEBFDF91CF911F910F91FF90EF90DF907C
:105AF000CF900895AF92BF92CF92DF92EF920F9323
:105B00001F93CF93DF93CDB7DEB76097CDBFDEBFD6
:105B10005C018A016630710509F086C0DA011296CF
:105B20008D919C911397BE016D5F7F4F0E94C222A1
:105B3000009709F479C0F80184819581BE01635F03
:105B40007F4F0E945422DC01CB010097A105B105D3
:105B500009F46AC0D80116968D919C911797BE01E1
:105B6000675F7F4F0E945422DC01CB010097A105A3
:105B7000B10509F459C0F80180859185BE016F5FB8
:105B80007F4F0E94C222009709F44EC0D8011A9696
:105B90008D919C911B97BE016B5F7F4F0E94542299
:105BA000DC01CB010097A105B105F1F1EDB7FEB71E
:105BB0003E97EDBFFEBF3196ADB7BEB71196AD9221
:105BC000BC9212978AEE96E2828393838B819C81AA
:105BD000848395838D859E858683978389859A8521
:105BE0008087918789819A81828793878D819E8121
:105BF000848795870E943D18EDB7FEB73E96EDBFAE
:105C0000FEBF4D855E856F85788909851A852B8550
:105C10003C85CD80DE808B81E9800E947113BC01C0
:105C2000C5010E941A191EC000D00F92ADB7BEB7B1
:105C30001196AD92BC9212978BEF96E213968D93CC
:105C40009C9314970E943D18EDB7FEB7A182B282D3
:105C50008FE297E2838394830E943D180F900F9008
:105C60000F900F906096CDBFDEBFDF91CF911F9157
:105C70000F91EF90DF90CF90BF90AF9008950F936A
:105C80001F93CF93DF930F920F92CDB7DEB78C01A6
:105C9000623071059CF0FA0182819381BE016F5FD1
:105CA0007F4F0E94C222009749F089819A810E9409
:105CB0005D13BC01C8010E941A1910C000D00F92D8
:105CC000EDB7FEB7018312838BE697E2838394835B
:105CD0000E943D180F900F900F900F900F900F9013
:105CE000DF91CF911F910F9108950F931F93CF9341
:105CF000DF930F92CDB7DEB78C01CE0101960E94E3
:105D00002D139C01E981E43040F4F0E0EE0FFF1F19
:105D1000EA5FFC4C8081918102C080E090E037FF17
:105D200005C041E552E28BEF95E202C04CE452E23D
:105D30006DB77EB76A5070406DBF7EBFEDB7FEB7DE
:105D40003196ADB7BEB711960D931C93129761E8CB
:105D500077E2628373834483558326833783808706
:105D600091870E943D186DB77EB7665F7F4F6DBF0C
:105D70007EBF0F90DF91CF911F910F9108950F93E8
:105D80001F93CF93DF938C01EA016230710574F1A8
:105D90008A819B816EE877E20E94C2160097D1F05B
:105DA0008A819B8162E977E20E94C2160097A1F086
:105DB0008A819B8165E977E20E94C216009771F0A3
:105DC0008A819B816BE977E20E94C216009771F489
:105DD00083E005C080E003C081E001C082E00E9452
:105DE0001D13BC01C8010E941A1910C000D00F92E7
:105DF000EDB7FEB7018312838FE997E28383948323
:105E00000E943D180F900F900F900F90DF91CF914F
:105E10001F910F910895CF93DF93EC010E94550CD1
:105E2000BC01CE010E941A19DF91CF910895CF9243
:105E3000DF92EF92FF920F931F93CF93DF93CDB733
:105E4000DEB7A197CDBFDEBF6C018B017A01CE0119
:105E5000019660E070E041E250E00E94AD1604302F
:105E6000110594F1F70182819381BE016F5F7F4F2D
:105E70000E94C721009709F45AC0F70106811781D3
:105E8000C80164EC77E20E94C216009791F0C80145
:105E900069EC77E20E94C216009771F0C8016DECC0
:105EA00077E20E94C216009709F041C041E050E03D
:105EB00005C043E050E002C042E050E0F7016481D9
:105EC0007581CE0101962CC00330110581F4F701D4
:105ED00082819381BE016F5F7F4F0E94C72100972F
:105EE00031F1F70164817581CE01019617C002304E
:105EF000110569F4F70182819381BE016F5F7F4FC5
:105F00000E94C721009799F0CE01019605C001308B
:105F1000110569F480E090E060E070E040E050E05E
:105F20000E94FB0BBC01C6010E941A1910C000D0D0
:105F30000F92EDB7FEB7C182D28281ED97E28383E3
:105F400094830E943D180F900F900F900F90A19690
:105F5000CDBFDEBFDF91CF911F910F91FF90EF90EA
:105F6000DF90CF9008958F929F92AF92BF92CF9281
:105F7000DF92EF92FF920F931F93CF93DF9300D0A6
:105F800000D0CDB7DEB74C018A011B821C821D8276
:105F90001E8219821A8263307105E4F0DA011296CA
:105FA0008D919C911397BE016D5F7F4F0E9454228B
:105FB000DC01CB010097A105B10509F446C0F80149
:105FC00084819581BE016F5F7F4F0E94C22200973E
:105FD000A1F43BC062307105C1F5DA0112968D91D2
:105FE0009C911397BE016D5F7F4F0E945422DC018C
:105FF000CB010097A105B10541F16B817C818D81B9
:106000009E8149810E94D20A5C010097C9F48AEFFF
:1060100090E00E941D464B815C816D817E81C9802C
:10602000DA8080914E3390914F3328E030E000E0E9
:1060300010E0E1E0EE2EF12C0E94A44497FD16C082
:10604000C401B5010E941A1929C000D00F92EDB702
:10605000FEB7818292828DEF97E2838394830E94C0
:106060003D180F900F900F900F9018C000D000D0E7
:10607000EDB7FEB73196ADB7BEB711968D929C9233
:10608000129727E238E222833383848395830E9428
:106090003D18EDB7FEB73696EDBFFEBF2696CDBFD5
:1060A000DEBFDF91CF911F910F91FF90EF90DF90B6
:1060B000CF90BF90AF909F908F900895CF93DF9334
:1060C000EC010E94FC0ABC01CE010E941A19DF916A
:1060D000CF9108952F923F924F925F926F927F924D
:1060E0008F929F92AF92BF92CF92DF92EF92FF92E8
:1060F0000F931F93CF93DF93CDB7DEB7A397CDBF99
:10610000DEBF7C018B010E943318009709F0AFC1FC
:106110000115110579F400D00F92ADB7BEB71196F5
:10612000ED92FC9212978CE598E213968D939C93D6
:10613000149710C0CE0101960E94F80B009789F0C9
:1061400000D00F92EDB7FEB7E182F2828CE698E2C2
:10615000838394830E943D180F900F900F900F90AF
:1061600086C100D00F92ADB7BEB71196ED92FC92EA
:10617000129785E096E213968D939C9314970E9454
:106180003D18EDB7FEB7E182F28289E898E2838399
:1061900094830E943D18ADB7BEB71196ED92FC9264
:1061A000129781EC98E213968D939C9314970E941A
:1061B0003D180F900F900F900F90AA24BB248824B5
:1061C000992419E0612E19E2712E09E2402E09E2AC
:1061D000502E81E4282E89E2382E41C1028113819C
:1061E0000A0D1B1DEDB7FEB77097EDBFFEBF3196D0
:1061F000ADB7BEB71196ED92FC9212976282738290
:10620000D80191968C9191978483158292968C9166
:1062100092978683178293968C91939780871186A5
:1062200094968C9194978287138695968C919597E6
:106230008487158696968C91868717860E943D18CE
:10624000EDB7FEB77096EDBFFEBFD8019E968D915B
:106250009C919F97009719F480E598E202C086E52B
:1062600098E2EDB7FEB73A97EDBFFEBF3196ADB7F6
:10627000BEB71196ED92FC921297428253828483AC
:106280009583D8019D968C919D97868317829796CA
:106290008D919C919897808791870E943D18F80175
:1062A00081A592A52DB73EB7265F3F4F2DBF3EBFBC
:1062B0003FEF80389307C9F000D000D0EDB7FEB7AC
:1062C0003196ADB7BEB71196ED92FC92129729E3C5
:1062D00039E222833383848395830E943D188DB7EE
:1062E0009EB706968DBF9EBF12C000D00F92ADB76D
:1062F000BEB71196ED92FC92129713962D923C9296
:1063000014970E943D180F900F900F900F90F80176
:1063100083A594A58230910559F18330910538F415
:10632000009781F08130910509F057C016C0843084
:106330009105A1F18430910530F18530910509F086
:106340004CC037C000D00F92ADB7BEB71196ED92DA
:10635000FC921297E7E4F9E236C000D00F92ADB795
:10636000BEB71196ED92FC921297E2E5F9E22BC0CE
:1063700000D00F92ADB7BEB71196ED92FC92129776
:10638000EDE5F9E220C000D00F92ADB7BEB711968F
:10639000ED92FC921297E8E6F9E215C000D00F9258
:1063A000ADB7BEB71196ED92FC921297E3E7F9E212
:1063B0000AC000D00F92ADB7BEB71196ED92FC9215
:1063C0001297EEE7F9E21396ED93FC9314970E946F
:1063D0003D180F900F900F900F90F3E0CF2ED12C1F
:1063E000CC0EDD1EC60160E070E041E250E00E948C
:1063F000AD16D80190964C91C601B80150E00E94AC
:10640000AA1600D000D0EDB7FEB73196ADB7BEB733
:106410001196ED92FC92129729E839E22283338398
:10642000C482D5820E943D180F900F90ADB7BEB7C1
:106430001196ED92FC92129785E096E213968D9359
:106440009C9314970E943D180894811C911CE0E3D2
:10645000F0E0AE0EBF1E0F900F900F900F90E981ED
:10646000FA8180819181881699060CF4B7CEA396A3
:10647000CDBFDEBFDF91CF911F910F91FF90EF90C5
:10648000DF90CF90BF90AF909F908F907F906F9054
:106490005F904F903F902F900895CF93DF93EC0142
:1064A000CB010097A9F400D00F92ADB7BEB71196FB
:1064B000CD93DC9312978CE899E213968D939C937D
:1064C00014970E943D180F900F900F900F901AC0D4
:1064D0000E942F1600D000D0EDB7FEB73196ADB7B1
:1064E000BEB71196CD93DC93129728EA39E2228346
:1064F0003383848395830E943D18EDB7FEB73696AB
:10650000EDBFFEBFDF91CF910895CF93DF93EC01F4
:10651000623071056CF0FA01828193816DE472E35F
:10652000AE010E94D510BC01CE010E941A1910C004
:1065300000D00F92EDB7FEB7818392838AEB99E288
:10654000838394830E943D180F900F900F900F90BB
:10655000DF91CF910895CF93DF93EC0188819981EA
:10656000009721F00E94BF0E18821982DF91CF910F
:1065700008950F931F93CF93DF938C01FC018281C9
:106580009381009721F0C80102960E94AB32F80176
:10659000808191810E94750EEC0197FD0EC068E527
:1065A00073E3A8010E94930DCE0162EE72E3A8018D
:1065B0000E94AC0DF801C283D383DF91CF911F916C
:1065C0000F910895AF92BF92CF92DF92EF92FF9218
:1065D0000F931F93CF93DF938C015B01EA01209708
:1065E00009F457C086E0C82ED12CC00ED11ECB01B5
:1065F000B60140E850E00E94170F7C01AE01481B35
:10660000590BC50160E070E00E94170FF7FC45C010
:10661000F80182819381009709F43FC0EE0DFF1DC0
:106620001582C60164EF7DE20E94FB160097A9F176
:10663000C60167EF7DE244E050E00E94BF1600977C
:1066400041F59801265F3F4FC901F90140812F5F55
:106650003F4F4C30C9F34A30B9F34D30A9F34930BC
:1066600099F34B3089F3403279F3DF0121912C30DB
:1066700051F02A3041F02D3031F0293021F02B300B
:1066800011F0203291F71C92F801628173810E940F
:10669000B840C80102960E94AB32DF91CF911F91A2
:1066A0000F91FF90EF90DF90CF90BF90AF90089543
:1066B000CF93DF9300D00F92CDB7DEB79C01CB0113
:1066C0004115510531F0BE016F5F7F4F0E94AB1045
:1066D00004C0C90102960E94AB322496CDBFDEBF32
:1066E000DF91CF9108950F931F93CF93DF938C0188
:1066F00086E890E00E948616EC01009739F180E070
:1067000090E060E070E00E943C0D8883998397FDE3
:1067100012C064E072E3A8010E94C50D009759F40D
:106720008881998161E070E049EB52E39E010E940B
:10673000F80D009759F088819981009711F00E9417
:10674000BF0ECE010E94A716C0E0D0E0CE01DF91BF
:10675000CF911F910F910895CF93DF93EC01029693
:106760000E94AB3288819981009711F00E94BF0E80
:10677000CE010E94A716DF91CF910895EF92FF926C
:106780000F931F93CF93DF93EC01CB017A01890123
:106790000E942F1600D000D0EDB7FEB73196ADB7EE
:1067A000BEB71196CD93DC9312972CEF3DE2228376
:1067B0003383848395830E943D180F920F92EDB727
:1067C000FEB73196ADB7BEB71196CD93DC93129755
:1067D00089E19EE282839383E482F58206831783B4
:1067E0000E943D188DB79EB708968DBF9EBFDF9162
:1067F000CF911F910F91FF90EF900895CF93DF936A
:10680000EC01888D998D1816190614F40E94BF0E9C
:106810008A8D9B8D009711F00E94701F8C819D8145
:106820000E94A716CE010E94A716DF91CF9108956E
:10683000CF92DF92EF92FF920F931F93CF93DF934C
:10684000EB010C811D81888999892A893B898217EE
:10685000930779F4EA85FB85309739F04C895D8997
:106860002E893F898C859D851995CE010E94FE3326
:106870007EC0EE80FF8088E090E0E80EF91E88E0A0
:10688000F80180831182128213828E859F850E9477
:106890007414F80184839583888999890E947414FB
:1068A000F80186839783970140E050E0BA010FC05A
:1068B000D080CC24818190E08C299D293296A0E063
:1068C000B0E0480F591F6A1F7B1F22503040223012
:1068D000310570F7C70196958795FC01EE0FFF1FF4
:1068E000E00FF11F880F991FE816F90641F090811B
:1068F00080E0A0E0B0E0480F591F6A1F7B1FCB016A
:10690000AA27BB2760707070480F591F6A1F7B1F32
:1069100060FF09C0CB01AA27BB2760707070480FC9
:10692000591F6A1F7B1FCA010E947414809590959D
:10693000F80182839383888D998DB801A7019E0108
:1069400000E010E00E9431108E159F0529F48C891B
:106950009D8901968C8B9D8B8A8D9B8D68EE73E053
:106960000E94AF1F888999890196888B998BDF9146
:10697000CF911F910F91FF90EF90DF90CF900895EE
:10698000AF92BF92CF92DF92EF92FF920F931F933D
:10699000CF93DF93EC016B018A01CA010E94831639
:1069A0007C010097A1F1C601B701A8010E94170F51
:1069B0006C018017910759F58CE1C816D10438F1A4
:1069C000F701808D918D0E9478142E853F85821766
:1069D0009307E9F48E899F8901968E8B9F8BA884FB
:1069E000B984A114B10499F00C84DD85C02DF701A0
:1069F000828D938D0E9478149C01A701445F5F4FA4
:106A0000F7010489CE01B60110E0F5011995C7011F
:106A10000E94A716DF91CF911F910F91FF90EF90E9
:106A2000DF90CF90BF90AF900895CF92DF92EF921A
:106A3000FF920F931F93CF93DF93EC016B01CA0179
:106A4000790101151105A1F40E942F162DB73EB74B
:106A50002A5030402DBF3EBFEDB7FEB73196ADB7DF
:106A6000BEB71196CD93DC9312972FE33EE213C08D
:106A700003301105F9F40E942F16ADB7BEB71A976F
:106A8000ADBFBEBFEDB7FEB731961196CD93DC9387
:106A900012972FE53EE222833383C482D582868318
:106AA0009783E086F1860E943D182DB73EB7265F9A
:106AB0003F4F20C00E942F16ADB7BEB71C97ADBF89
:106AC000BEBFEDB7FEB731961196CD93DC9312970A
:106AD0002CE93EE222833383C482D5828683978366
:106AE000E086F186028713870E943D182DB73EB7D6
:106AF000245F3F4F2DBF3EBFDF91CF911F910F917C
:106B0000FF90EF90DF90CF9008954F925F926F9239
:106B10007F928F929F92AF92BF92CF92DF92EF922D
:106B2000FF920F931F93CF93DF930F920F92CDB7E6
:106B3000DEB75C013B01490168018CE190E04983CB
:106B40005A830E9486162C0149815A81009709F4C4
:106B500042C08A01C80108960E948616F201848309
:106B600095830097A9F182E090E061E070E00E94D7
:106B70003C0DF201808F918F181619064CF560ECD0
:106B800074E3A2010E94AC0DF50180819181A28184
:106B9000B381F20180839183A283B383628A738A73
:106BA000068317831686178680869186C286D386CB
:106BB000E486F58680E090E060E070E048E154E330
:106BC00092010E94C21FF201828F938F009731F4CD
:106BD000C2010E94FE338DEF9FEF02C080E090E083
:106BE0000F900F90DF91CF911F910F91FF90EF9039
:106BF000DF90CF90BF90AF909F908F907F906F90DD
:106C00005F904F9008954F925F926F927F928F9214
:106C10009F92AF92BF92CF92DF92EF92FF920F932B
:106C20001F93CF93DF9300D00F92CDB7DEB72C0127
:106C30005B016A018091043290910532A091063285
:106C4000B091073289839A83AB83BC83E1E0EE2E57
:106C5000F12CF0E26F2E712C13E0812E912C49C0A3
:106C60008701000F111F0C0D1D1DD8018D919C91E6
:106C70006BEC7EE20E94C216009791F40894E11C2E
:106C8000F11CEA14FB040CF081C0F701EE0FFF1FAA
:106C9000EC0DFD1D808191810E941B544C0126C08A
:106CA000F801808191816EEC7EE20E94C21600970D
:106CB00091F40894E11CF11CEA14FB040CF066C08A
:106CC000F701EE0FFF1FEC0DFD1D808191810E94E9
:106CD0001B543C010BC0D8018D919C91BE016F5F8C
:106CE0007F4F0E94AA14009709F450C00894E11C39
:106CF000F11CEA14FB040CF4B3CF89819A81AB81B7
:106D0000BC814091043250910532609106327091FD
:106D1000073284179507A607B707C1F1CE01019680
:106D2000B401A30125E135E30EEB13E372010E94E8
:106D300085358C0197FD05C084ECE82E8EE2F82E97
:106D400004C0B7ECEB2EBEE2FB2EC8010E944C1F24
:106D5000EDB7FEB73A97EDBFFEBF3196ADB7BEB700
:106D600011964D925C92129721ED3EE2228333837D
:106D7000E482F58206831783808791870E943D18FD
:106D8000EDB7FEB73A96EDBFFEBF14C000D00F922C
:106D9000ADB7BEB711964D925C9212978EED9EE202
:106DA00013968D939C9314970E943D180F900F900B
:106DB0000F900F902496CDBFDEBFDF91CF911F9132
:106DC0000F91FF90EF90DF90CF90BF90AF909F908A
:106DD0008F907F906F905F904F900895AF92BF9289
:106DE000CF92DF92EF92FF920F931F93CF93DF9397
:106DF000EC01B62EA72E88899989009769F02C811D
:106E00003D818E819F81289FA001299F500D389F31
:106E1000500D11246A0104C0CA88DB88EC88FD8803
:106E20006C857D85888599850E94D520EA8DFB8DAE
:106E3000309749F08C0120E030E08C8D9D8D6B2DDA
:106E40007A2DA60119958A819B810E94A7168881B7
:106E500099810E94BF0E88899989009721F48E89B3
:106E60009F890E94BF0ECE010E94A7168B2D9A2DDE
:106E7000DF91CF911F910F91FF90EF90DF90CF9016
:106E8000BF90AF9008958F929F92AF92BF92CF9292
:106E9000DF92EF92FF920F931F93CF93DF93EC015A
:106EA0005B014A016801790100D00F92ADB7BEB70E
:106EB00011968D939C9312978FE09FE213968D937A
:106EC0009C9314970E943D180F900F900F900F9075
:106ED000A114B104E9F0C5010E944C1FEDB7FEB743
:106EE0003897EDBFFEBF3196ADB7BEB71196CD93C3
:106EF000DC93129722E13FE222833383A482B5829E
:106F0000868397830E943D18EDB7FEB738964DC033
:106F1000C114D104E104F10491F12DB73EB72E5014
:106F200030402DBF3EBF0DB71EB70F5F1F4FADB72F
:106F3000BEB71196CD93DC93129785E29FE2F801DC
:106F40008283938384829582C682D782E086F1868B
:106F5000B401882777FD8095982FA70196010E949C
:106F60007E50F80122873387448755870E943D1859
:106F70002DB73EB7225F3F4F2DBF3EBF18C000D098
:106F800000D0EDB7FEB73196ADB7BEB71196CD9331
:106F9000DC93129787E59FE28283938384829582B4
:106FA0000E943D18EDB7FEB73696EDBFFEBFDF91EC
:106FB000CF911F910F91FF90EF90DF90CF90BF90F6
:106FC000AF909F908F9008950F931F93CF93DF936F
:106FD0008C01EB0100D00F92EDB7FEB78183928355
:106FE0008DE79FE2838394830E943D180F900F905A
:106FF0000F900F901C161D06BCF4CE0160E570E0EA
:107000000E946B50009781F400D00F92EDB7FEB74D
:10701000018312838FE09FE2838394830E943D1853
:107020000F900F900F900F90DF91CF911F910F91C4
:107030000895CF93DF93EC01CB010E94750EBC0144
:107040008E8B9F8B97FF04C0CE010E94EE3614C03A
:1070500066E878E3AE010E94930D8E899F896FE305
:1070600078E3AE010E94AC0D0E940D20A0E0B0E0DC
:1070700088879987AA87BB87DF91CF910895CF939F
:10708000DF93EC019B01888999890097E1F541150F
:10709000510561F40E940D20A0E0B0E08C879D872F
:1070A000AE87BF87CE0160E070E00BC06A817B8154
:1070B0004C815D81C9010E94170FBC0197FF04C07C
:1070C000CE010E94EE361FC02E813F812F5F3F4FC1
:1070D0002E833F83CB01AA2797FDA095BA2F4A891B
:1070E0005B896C897D89480F591F6A1F7B1F4A8BFA
:1070F0005B8B6C8B7D8BE88DF98D309721F08C8DBF
:107100009D8DB9011995DF91CF910895EF92FF926E
:107110000F931F93CF93DF93EC014115510519F4A1
:107120006CEF7FEF3CC00E940D20A0E0B0E08887AC
:107130009987AA87BB87EE24FF2421C06A817B81BF
:10714000600F711F401B510B888199810E94CD0FE8
:10715000BC0197FD0BC0080F191F02C000E010E032
:107160004C815D810417150748F322C0CE0117C07A
:107170008C8D9D8DB70119950894E11CF11C8E81B1
:107180009F81E816F90650F30E940D20A0E0B0E0C0
:107190008C879D87AE87BF87CE0160E070E00E943C
:1071A000EE36DF91CF911F910F91FF90EF900895F0
:1071B000E88DF98D3097E1F6DFCF4F925F926F92B5
:1071C0007F928F929F92AF92BF92CF92DF92EF9277
:1071D000FF920F931F93CF93DF932C013B01EA01A2
:1071E00059014801209709F456C02115310509F4C9
:1071F00052C06115710509F44EC08EE190E00E9405
:1072000086168C01009709F449C0FC01C683D78318
:10721000A482B582808E918EE28EF38EC48ED58E3E
:1072200081E090E0808B918BC5010E948316F8016C
:1072300082839383009721F4C8016DEF7FEF0DC027
:1072400080E090E060E070E00E943C0DBC01F8013D
:107250008083918397FF04C0C8010E94EE3620C04E
:10726000B201A3010E94330EBC0197FDF5CFF801D6
:107270008081918166E878E3A8010E94930DF8016E
:10728000808191816FE378E3A8010E94AC0DF80141
:107290008081918105C08EEF9FEF02C08DEF9FEF3F
:1072A000DF91CF911F910F91FF90EF90DF90CF90E2
:1072B000BF90AF909F908F907F906F905F904F9016
:1072C00008958F929F92AF92BF92CF92DF92EF92EA
:1072D000FF920F931F93CF93DF934C017B015A01D1
:1072E00069018EE190E00E948616EC01009719F486
:1072F00080E090E010C0EC82FD82A88EB98ECA8E2C
:10730000DB8E0C8F1D8FC7010E9483168A839B839F
:10731000009731F4CE016DEF7FEF0E94EE3623C06F
:1073200080E090E060E070E00E943C0DBC0188834A
:10733000998397FD14C064E072E3A4010E94C50D17
:10734000BC0197FD0CC08881998161E070E049E142
:1073500058E39E010E94F80DBC0197FF02C0CE01C8
:10736000DCCF88819981DF91CF911F910F91FF90A0
:10737000EF90DF90CF90BF90AF909F908F90089547
:107380002F923F924F925F926F927F928F929F9235
:10739000AF92BF92CF92DF92EF92FF920F931F9323
:1073A000CF93DF9300D000D0CDB7DEB74C015B01A7
:1073B0006A018091043290910532A0910632B09119
:1073C000073289839A83AB83BC8322243324412CE4
:1073D00024E0522E20E034E02D833E83E8E86E2E38
:1073E000E3E17E2EF1E0EF2EF12C7DC08701000F4E
:1073F000111F0C0D1D1DD8018D919C916FE77FE22F
:107400000E94C216009791F40894E11CF11CEA1442
:10741000FB040CF007C1F701EE0FFF1FEC0DFD1D83
:10742000808191810E941B543C015AC0F8018081E7
:10743000918162E87FE20E94C216009799F4089455
:10744000E11CF11CEA14FB040CF0ECC0F701EE0F98
:10745000FF1FEC0DFD1D808191810E941B548D83C7
:107460009E833EC0D8018D919C9165E87FE20E9489
:10747000C216009791F40894E11CF11CEA14FB0475
:107480000CF0D0C0F701EE0FFF1FEC0DFD1D808149
:1074900091810E941B542C0123C0F80180819181AD
:1074A00068E87FE20E94C2160097A1F0D8018D9192
:1074B0009C916BE87FE20E94C216009779F0F80178
:1074C00080819181BE016F5F7F4F0E94AA14009757
:1074D00039F4A8C0F1E02F2E312C02C0222433242D
:1074E0000894E11CF11CEA14FB040CF47FCF211476
:1074F000310411F189819A81AB81BC8140910432C0
:1075000050910532609106327091073284179507C9
:10751000A607B70709F486C0CE010196B3014D81D5
:107520005E81920104EE17E3E3E4EE2EE7E3FE2E24
:1075300064010E94DD3809C0C301B20144EE57E383
:1075400023E437E384010E9461398C0197FF1EC058
:107550000E944C1F2DB73EB72A5030402DBF3EBF72
:10756000EDB7FEB73196ADB7BEB711968D929C922E
:1075700012972EE83FE2228333832BE93FE22483F4
:107580003583068317838087918744C02114310493
:1075900059F1CE0101960E942F162DB73EB72E50FD
:1075A00030402DBF3EBFEDB7FEB73196ADB7BEB789
:1075B00011968D929C9212972FE93FE2228333839A
:1075C00084839583668277822D813E8120873187EF
:1075D00042865386048715870E943D188DB79EB753
:1075E0000E968DBF9EBF32C0ADB7BEB71A97ADBF66
:1075F000BEBFEDB7FEB7319611968D929C92129751
:1076000080ED9FE2828393836482758246825782F3
:10761000008711870E943D18EDB7FEB73A96EDBF7F
:10762000FEBF14C000D00F92ADB7BEB711968D92B9
:107630009C9212978BEF9FE213968D939C931497D5
:107640000E943D180F900F900F900F902696CDBF7F
:10765000DEBFDF91CF911F910F91FF90EF90DF90F0
:10766000CF90BF90AF909F908F907F906F905F90E2
:107670004F903F902F900895CF93DF93EC018C8132
:107680009D811816190614F40E94BF0E8E819F81E9
:10769000009711F00E94701FCE010E94A716DF9183
:1076A000CF910895CF93DF93EB01E881F981309773
:1076B00039F08A819B8160E070E04FEE5FEF1995B1
:1076C000CE010E943C3BDF91CF9108950F931F9311
:1076D000CF93DF938C01DB01EA01109711F5CA010A
:1076E0000E944C1F2DB73EB7285030402DBF3EBFE3
:1076F000EDB7FEB73196ADB7BEB711960D931C939B
:1077000012972CE230E32283338384839583C683EC
:10771000D7830E943D18CDB7DEB72896CDBFDEBF18
:107720003AC02DB73EB7205130402DBF3EBFEDB718
:10773000FEB73196CDB7DEB789839A838CE490E3A8
:107740008283938315968D919C9116978459984FB7
:107750008483958314968C91149790E00196868388
:10776000978313968C9113978087118612968C912C
:1077700012978287138611968C91119784871586AC
:107780008C91868717860E943D182DB73EB7205FE3
:107790003F4F2DBF3EBFDF91CF911F910F910895B5
:1077A0008F929F92AF92BF92CF92DF92EF92FF9211
:1077B0000F931F93CF93DF93CDB7DEB7E097CDBF85
:1077C000DEBF4C018B015A01CE01019660E070E0F2
:1077D00040E350E00E94AD1683E2898388E090E0A8
:1077E0000E9486167C01009709F443C081E090E076
:1077F00060E070E00E943C0D6C01181619068CF5D3
:10780000F70100831183A282B3828483958388E881
:1078100093E160E070E042E55BE397010E94C21FE4
:10782000F701868397830097E1F0C601B4014BE727
:1078300050E00E94330E8C010097B9F4C6016CEF42
:107840007EE3A7010E94AC0D97FD0EC0C601BE01EC
:107850006F5F7F4F40E350E00E94CD0F97FF0BC05A
:1078600003C00DEF1FEF01C08C01C7010E943C3B1C
:1078700002C00DEF1FEFC801E096CDBFDEBFDF9164
:10788000CF911F910F91FF90EF90DF90CF90BF901D
:10789000AF909F908F900895CF92DF92EF92FF92DA
:1078A0000F931F93CF93DF9300D00F92CDB7DEB726
:1078B0007C01623071050CF440C0DA0112968D91A2
:1078C0009C911397BE016F5F7F4F0E94AA1400978F
:1078D000A1F1CE01019666E67BE3A7010E94D03BB1
:1078E0008C0197FD05C096E7C92E90E3D92E04C000
:1078F00089E7C82E80E3D82EC8010E944C1FEDB73F
:10790000FEB73A97EDBFFEBF3196ADB7BEB7119641
:10791000ED92FC9212972DE730E322833383C482E9
:10792000D58206831783808791870E943D18EDB723
:10793000FEB73A96EDBFFEBF14C000D00F92ADB7B0
:10794000BEB71196ED92FC9212978AE890E31396D7
:107950008D939C9314970E943D180F900F900F9059
:107960000F902496CDBFDEBFDF91CF911F910F9175
:10797000FF90EF90DF90CF9008954F925F926F92BB
:107980007F928F929F92AF92BF92CF92DF92EF92AF
:10799000FF920F931F93CF93DF93CDB7DEB7C454FD
:1079A000D040CDBFDEBF8B01DE011196E4EAF0E3EB
:1079B00024E301900D922150E1F7DC016D917D915E
:1079C0008D919C9120E831E541E050E00E947E508D
:1079D0002DAB3EAB4FAB58AF20E13EE040E050E076
:1079E0000E94A050F80122832CE330E040E050E0F8
:1079F0000E94A050D80111962C9311976C936DA9F9
:107A00007EA98FA998AD6C5F7F4F8F4F9F4F27E066
:107A100030E040E050E00E94A050F8016187A2EB06
:107A20004A2EA7E05A2E612C712C2BC16DA97EA97C
:107A30008FA998AD2DE631E040E050E00E94A050C3
:107A400073016201C20ED31EE41EF51EDC01CB01E0
:107A50008827B7FD83959927AA27BB27C81AD90A73
:107A6000EA0AFB0A2196CCAEDDAEEEAEFFAE219760
:107A700053014201089481089108A108B108A701A7
:107A80009601215030404040504025962CAF3DAFEC
:107A90004EAF5FAF2597C501B40124E030E040E070
:107AA00050E00E94A050DC01CB018827B7FD8395F0
:107AB0009927AA27BB2769017A01C81AD90AEA0AB5
:107AC000FB0AC9AEDAAEEBAEFCAEC501B40124E6EA
:107AD00030E040E050E00E94A0506B017C01CC24DB
:107AE000F7FCC394DD24EE24FF24C501B4012CE986
:107AF0003FEF4FEF5FEF0E94A050C20ED31EE41E77
:107B0000F51E29AD3AAD4BAD5CAD2C0D3D1D4E1DA6
:107B10005F1D29AF3AAF4BAF5CAFC501B40120E99F
:107B200031E040E050E00E94A050DC01CB0188270A
:107B3000B7FD83959927AA27BB2769017A01C81A3F
:107B4000D90AEA0AFB0AD701C601C9ACDAACEBAC28
:107B5000FCACC80ED91EEA1EFB1EC9AEDAAEEBAEF7
:107B6000FCAE25966CAD7DAD8EAD9FAD259720E921
:107B700031E040E050E00E94A0506B017C01CC2439
:107B8000F7FCC394DD24EE24FF2425966CAD7DAD77
:107B90008EAD9FAD259720E73EEF4FEF5FEF0E9440
:107BA000A050C20ED31EE41EF51E25966CAD7DAD11
:107BB0008EAD9FAD259724E630E040E050E00E9476
:107BC000A05049015A01DC01CB018827B7FD8395FC
:107BD0009927AA27BB27881A990AAA0ABB0A2596B9
:107BE0006CAD7DAD8EAD9FAD259724E030E040E0DB
:107BF00050E00E94A050DC01CB018827B7FD83959F
:107C00009927AA27BB27821B930BA40BB50B880EC1
:107C1000991EAA1EBB1EC80CD91CEA1CFB1CC30162
:107C2000B20121962CAD3DAD4EAD5FAD2197621BEB
:107C3000730B840B950B2DE631E040E050E00E9481
:107C40004050DC01CB01C80ED91EEA1EFB1E89ADD7
:107C50009AADABADBCAD8C0D9D1DAE1DBF1DCDA8AD
:107C6000DEA8EFA8F8ACC80ED91EEA1EFB1ECDAAEE
:107C7000DEAAEFAAF8AE21964CAC5DAC6EAC7FAC40
:107C80002197CDA8DEA8EFA8F8ACF7FCCFCE23E073
:107C9000C22ED12CE12CF12CC420D520E620F720D7
:107CA000C114D104E104F104E1F4C301B20124E6FA
:107CB00030E040E050E00E94A050DC01CB01009792
:107CC000A105B10599F4C301B20120E931E040E01A
:107CD00050E00E94A050DC01CB010097A105B10546
:107CE00029F08DE691E0A0E0B0E004C08EE691E0DE
:107CF000A0E0B0E02DA93EA94FA958AD281739073B
:107D00004A075B070CF092CEC2018C569740D8010F
:107D100015968D939C93169717962D933C931897D1
:107D2000C114D104E104F104F9F4C301B20124E661
:107D300030E040E050E00E94A050DC01CB01009711
:107D4000A105B105A1F4C301B20120E931E040E091
:107D500050E00E94A050AB01BC0181E090E04115D1
:107D600051056105710529F080E090E002C081E0D5
:107D700090E02AE130E0829FF001839FF00D929F16
:107D8000F00D1124EC0FFD1F79964BE050E060E000
:107D900070E004C041505040604070409291829128
:107DA000A0E0B0E0CDA8DEA8EFA8F8ACC816D906D0
:107DB000EA06FB067CF3F8014483C81AD90AEA0AEA
:107DC000FB0AD701C6018F5F838381E090E0CC5B23
:107DD000DF4FCDBFDEBFDF91CF911F910F91FF909D
:107DE000EF90DF90CF90BF90AF909F908F907F905B
:107DF0006F905F904F900895AF92BF92CF92DF92B5
:107E0000EF92FF920F931F93CF93DF93CDB7DEB71F
:107E10006097CDBFDEBF5C016B018A014033510525
:107E200080F1CA010E9483167C01009779F1C60196
:107E3000B701A8010E94170FAC018017910741F507
:107E4000D70190966D917D918D919C9193974F87DD
:107E5000588B0E94A714DC01CB0180589E47AA4A88
:107E6000B34889839A83AB83BC83F894CE0101968F
:107E7000BE016B5F7F4F0E94BD3C78944F8558894F
:107E800007C040EF5FEFEE24FF2402C04DEF5FEF2D
:107E9000D501ED91FC911197309741F012968D919B
:107EA0009C911397BE016B5F7F4F1995C7010E948C
:107EB000A716C5010E943C3B6096CDBFDEBFDF9197
:107EC000CF911F910F91FF90EF90DF90CF90BF90D7
:107ED000AF900895CF92DF92EF92FF920F931F938E
:107EE000CF93DF936C018B01CB010E94B3167C0111
:107EF000C0E0D0E00DC0B8016C0F7D1FA7014C1B86
:107F00005D0BC6010E94CD0F97FD07C0C80FD91F9A
:107F1000CE15DF0584F380E090E0DF91CF911F91D3
:107F20000F91FF90EF90DF90CF9008958F929F92E6
:107F3000AF92BF92CF92DF92EF92FF920F931F9377
:107F4000CF93DF934C015B016A0180E490E00E94D3
:107F500083167C0100E010E01DC0E601C01BD10BC0
:107F6000C134D10514F0C0E4D0E0B501600F711F39
:107F7000C701AE010E944154C401B701AE010E9485
:107F8000CD0FEC0197FF04C0C7010E94A7160AC0DD
:107F9000080F191F0C151D0504F3C7010E94A71631
:107FA000C0E0D0E0CE01DF91CF911F910F91FF9003
:107FB000EF90DF90CF90BF90AF909F908F900895FB
:107FC0000F931F93CF93DF938C01EB01CB010E94A2
:107FD0004A54AC01C801BE010E94963FDF91CF9187
:107FE0001F910F910895EF92FF920F931F93CF93DC
:107FF000DF93CDB7DEB76C97CDBFDEBF8C018EE4CB
:108000009FE2A1E4B0E08B879C87AD87BE87FE012D
:108010003F968EE0DF011D928A95E9F70115110563
:1080200009F499C0C8016FE078E00E94E03F9C012C
:1080300097FD93C0CE01019660E070E040E050E013
:1080400020E030E00E946C0C009731F4CE010196E4
:108050000E942F167C0104C085EFE82E80E3F82EE5
:10806000C80169E67AE00E94E03F9C0197FD75C077
:10807000C801B7010E946A3F9C0197FD6EC0C8010C
:108080006EE77AE00E94E03F9C0197FD66C0CE015A
:1080900005960E94C60C009789F58DB79EB742974A
:1080A0008DBF9EBFEDB7FEB73196CE010B96ADB733
:1080B000BEB711968D939C93129782E190E08283D4
:1080C000938389EF90E3848395838D8186831782E0
:1080D0008E81808711868F81828713868885848729
:1080E00015868985868717868A85808B118A0E94E6
:1080F0006C558DB79EB742968DBF9EBFC80169E98A
:108100007AE00E94E03F9C0197FD27C0C801BE01B4
:10811000655F7F4F0E946A3F9C0197FD1EC0C801AA
:108120006FEA7AE00E94E03F9C0197FD16C0C8010B
:108130006AEC7AE00E94E03F9C0197FD0EC0C80106
:108140006FEE7CE00E94E03F9C01181619062CF4AB
:1081500020E030E002C02FEF3FEFC9016C96CDBFA9
:10816000DEBFDF91CF911F910F91FF90EF900895A7
:10817000EF92FF920F931F93CF93DF930F920F9283
:10818000CDB7DEB78C017B0167E171E30E94C216B7
:10819000009709F471C0C80169E171E30E94C21639
:1081A000009709F469C0C8016CE171E34CE050E04C
:1081B0000E94BF16009709F058C000D000D0EDB75C
:1081C000FEB73196045F1F4FADB7BEB711960D9342
:1081D0001C93129789E291E382839383CE010196E7
:1081E000848395830E94A3552DB73EB72A5F3F4FE6
:1081F0002DBF3EBF009709F43FC089819A8183302B
:10820000910511F1843091054CF481309105B1F064
:1082100082309105B4F4009771F02EC0853091053D
:10822000C9F0853091059CF086309105B1F087301A
:10823000910511F515C080E290E014C081E290E054
:1082400011C082E290E00EC083E290E00BC084E2B5
:1082500090E008C085E290E005C086E290E002C0B0
:1082600087E290E00E94DD4507C0C80166E371E344
:108270000E94C216009729F4C7010E94F33F9C0197
:1082800028C0C80162E471E30E94C216009781F41D
:10829000C70164EF71E00E94E03F9C0197FD19C0A7
:1082A000C70160E372E045EE54E00E94963F08C0CB
:1082B000E114F10461F0C70165E177E00E94E03F5D
:1082C0009C01181619062CF420E030E002C02FEFB4
:1082D0003FEFC9010F900F90DF91CF911F910F9148
:1082E000FF90EF9008950F931F93CF938C01C62FAB
:1082F000BA0180E090E026E631E040E050E00E94E4
:10830000405020914C3330914D3340E050E00E947A
:108310007E5020934A3330934B332FB7F894F801B3
:10832000308181E090E002C0880F991FCA95E2F782
:10833000880F880F832B80832FBFCF911F910F91C0
:1083400008950F931F93CF93DF93CDB7DEB72A978E
:10835000CDBFDEBFBE016C5F7F4F87E0FB01119296
:108360008A95E9F78E010F5F1F4F83E0F8011192A4
:108370008A95E9F786E0888781E08E8380E092E045
:108380000E944E4B80E092E063E771E40E94234C30
:1083900019821A828B81807F81608B8380E092E0DA
:1083A00060E0A8010E94B34B82E06FE270E00E949F
:1083B000C246182F00E082E06EE270E00E94C246E2
:1083C00090E0802B912B80934C3390934D3380E041
:1083D00092E00E941D4B9FB7F894E0E0F2E08081AC
:1083E000846080839FBF2A96CDBFDEBFDF91CF918F
:1083F0001F910F91089580914A3390914B33815191
:108400009140089500D000D0EDB7FEB73196ADB7DA
:10841000BEB711968D939C9312978CE491E382835F
:108420009383648375830E943D188DB79EB706962B
:108430008DBF9EBF08950E94D8450E9414200895C4
:108440006115710529F08FB7F89480935233089520
:10845000809152338FBF0895662349F000D00F9268
:10846000EDB7FEB7818392838EE591E308C000D01B
:108470000F92EDB7FEB7818392838AE791E38383FE
:1084800094830E943D180F900F900F900F900895C5
:10849000CF93DF93EC01CB01009761F500D00F92F1
:1084A000ADB7BEB71196CD93DC93129784E991E3F3
:1084B00013968D939C9314970E943D18809150338E
:1084C000909151330F900F900F900F90009709F4F7
:1084D00049C00E94AC33109250331092513300D0F7
:1084E0000F92EDB7FEB7C183D28386EA91E383830F
:1084F000948332C00E942F1600D000D0EDB7FEB793
:108500003196ADB7BEB71196CD93DC93129726EB9B
:1085100031E322833383848395830E943D18EDB732
:10852000FEB73696EDBFFEBF80E590E00E94733344
:1085300080935033909351330097A1F000D00F9265
:10854000ADB7BEB71196CD93DC93129786EC91E34D
:1085500013968D939C9314970E943D180F900F9043
:108560000F900F90DF91CF9108958EE290E061150A
:10857000710539F00E94AD468EE190E00E941D46E3
:1085800008950E9498460895AF92BF92CF92DF92CD
:10859000EF92FF920F931F93CF93DF93CDB7DEB788
:1085A000AB97CDBFDEBF1A820E94F44580E490E015
:1085B0006BE172E40E94AF450E94601F97FDB4C159
:1085C00080EA99E040E052EC61E070E028E030E0C1
:1085D00000E010E0E1E0EE2EF12CCC24DD240E943E
:1085E000A44497FDA1C180E090E067E375E440EA10
:1085F00059E024E030E00E943F1D5C01009709F43F
:1086000093C10E94492180EA9BE040E052EC61E086
:1086100070E028E030E00E94A44497FD85C180E02E
:1086200090E060E275E447E355E420E232E400EADA
:108630001BE00E940F0A97FD77C180EA9BE08093C0
:108640004E3390934F330E94A14185EB92E4B501E4
:108650000E94900ACE0102960E94710ACE010196F4
:108660000E942D1382E092E4B5010E94EC0B88E495
:1086700092E4B5010E94BD0C8CE292E4B5010E9427
:108680001914C50164EF72E340E050E00E94241821
:10869000C5016EEE72E340E050E00E942418C5016F
:1086A00064EC72E340E050E00E942418C5016EEBD8
:1086B00072E340E050E00E942418C50168EB72E3C9
:1086C00040E050E00E942418C50162EB72E340E0F4
:1086D00050E00E942418C5016CEA72E340E050E0CB
:1086E0000E942418C50166EA72E340E050E00E944F
:1086F0002418C50160EA72E340E050E00E942418AB
:10870000C5016AE672E340E050E00E942418C5010A
:108710006AE972E340E050E00E942418C50164E970
:1087200072E340E050E00E942418C5016EE872E355
:1087300040E050E00E942418C50168E872E340E080
:1087400050E00E942418C50162E872E340E050E066
:108750000E942418C5016CE772E340E050E00E94DB
:108760002418C50166E772E340E050E00E94241837
:10877000C50160E772E340E050E00E942418C501A3
:108780006EE572E340E050E00E942418C50168E500
:1087900072E340E050E00E942418C50162E572E3F4
:1087A00040E050E00E942418C50168EE72E340E00A
:1087B00050E00E942418C50162EE72E340E050E0F0
:1087C0000E942418C5016CED72E340E050E00E9465
:1087D0002418C50166ED72E340E050E00E942418C1
:1087E000C5016AEC72E340E050E00E942418C50124
:1087F00060E073E340E050E00E942418C5016AEF96
:1088000072E340E050E00E942418C50164E672E380
:1088100040E050E00E942418C5016CE472E340E09F
:1088200050E00E942418C50166E472E340E050E085
:108830000E942418C50160E472E340E050E00E9409
:108840002418C50164E173E340E050E00E9424185D
:10885000C5016AE173E340E050E00E942418C501BD
:108860006EE073E340E050E00E942418C50168E028
:1088700072E340E050E00E94241889818823B1F51A
:1088800066E172E088EA90EC0E947C14DC01CB0186
:108890008F839887A987BA8760E07FEF8FEF9FEF7C
:1088A0000E947C14DC01CB018B839C83AD83BE834F
:1088B000CE010B9666ED71E30E94C51686ED91E33D
:1088C0000E94B3168BA7CE010B9661EE71E340E0D8
:1088D00050E00E94FB0BCE010796BE016D5F7F4FFB
:1088E00040E050E020E030E00E94630C80EA99E034
:1088F0000E945C45009751F080EA99E060E070E0EA
:108900000E940845682FC5010E94A91A8A8180FF2C
:1089100006C08DE290E00E947D46009711F40E940F
:108920001E110E944420E2CF8FEF9FEFAB96CDBF88
:10893000DEBFDF91CF911F910F91FF90EF90DF90FD
:10894000CF90BF90AF900895AF92BF92CF92DF9239
:10895000EF92FF920F931F93CF935C01C114D10448
:1089600009F044C0265030402430310528F4205E00
:108970003C4CF901C08101C0C0E00130110539F063
:108980000130110538F00230110581F502C0C062D6
:1089900001C0C063F2E0EF16F10409F4C8609A0167
:1089A000AB0184E0220F331F441F551F8A95D1F776
:1089B000213088E4380788EE480781E0580750F4F2
:1089C00060E078E488EE91E00E947E5021503040D3
:1089D00088E103C02FEF3FEF8CE1F5011482C583DE
:1089E00026833783848380E090E002C086EF9FEF88
:1089F000CF911F910F91FF90EF90DF90CF90BF909C
:108A0000AF900895FC01818185FFFDCF60830895BB
:108A10000F931F93CF93DF93EC018B010E940D20E6
:108A20000115110531F4898187FFFDCF888190E020
:108A300002C086EF9FEFDF91CF911F910F910895B4
:108A4000DC0180E090E00EC011962C91119727FF79
:108A5000FBCF2C916115710521F0FB01E80FF91F87
:108A600020830196841795077CF3CA010895CF925D
:108A7000DF92EF92FF920F931F93CF93DF936C01DE
:108A80007A018B01C0E0D0E00AC0F80161918F014A
:108A9000772767FD7095C6010E9402452196CE1585
:108AA000DF059CF3C701DF91CF911F910F91FF90DC
:108AB000EF90DF90CF900895FC01818190E0807865
:108AC000907008958530910540F4FC01EE0FFF1F72
:108AD000EC5DFC4C8081918108958FEE91E30895C7
:108AE000CF92DF92EF92FF926B017C01E0915333C2
:108AF000F0915433309709F0199580915533909146
:108B00005633A0915733B09158338C0D9D1DAE1D37
:108B1000BF1DBC01CD010E94FF47FF90EF90DF9089
:108B2000CF9008958093593390935A339C01B901A3
:108B3000882777FD8095982F28EE33E040E050E0BD
:108B40000E9440500E947E502093553330935633FC
:108B5000409357335093583380E090E00895CF927C
:108B6000DF92EF92FF926C01609353337093543312
:108B70000E941F4880E795E40E941A48C6010E949F
:108B80009245C0905533D0905633E0905733F090D3
:108B900058330E94DA476C0D7D1D8E1D9F1D0E946B
:108BA000FF4780E090E0FF90EF90DF90CF90089536
:108BB0008091593390915A330895CF93DF93EC010C
:108BC0000E947D46009721F0CE010E94AD4603C071
:108BD000CE010E949846DF91CF9108950E94984659
:108BE00008950E94AD46089587E0E0EAF0E08283B0
:108BF0000E94CC460E94234780EA96E068E040E06D
:108C000053E00E94924780EA96E064E040E050E042
:108C10000E94924783E090E060E10E94F54684E084
:108C200090E060E10E94F54686E090E060E10E94FD
:108C3000F546789480E090E008959C0108C08FE3A9
:108C40009FE10197F1F700C000002150304021154D
:108C50003105A9F70895CF93C82F8A3031F480EAFF
:108C600099E06DE070E00E9402456C2F772767FD68
:108C7000709580EA99E00E940245CF9108958BE5B6
:108C800093E3089580E090E0089560FF18C0282FD6
:108C900026952695269530E0205D3F4F877061E050
:108CA00070E002C0660F771F8A95E2F7C90155E0B0
:108CB000880F991F5A95E1F740E050E019C061FF15
:108CC00019C0282F26952695269530E0205D3F4F28
:108CD000877061E070E002C0660F771F8A95E2F747
:108CE000C90145E0880F991F4A95E1F740E051E03E
:108CF0000E94924780E090E00895E82FE695E6957F
:108D0000E695F0E0F09665E0EE0FFF1F6A95E1F75B
:108D10004085877021E030E002C0220F331F8A9522
:108D2000E2F7422381E090E011F480E090E00895C2
:108D3000E82FE695E695E695F0E0F09675E0EE0F03
:108D4000FF1F7A95E1F7877021E030E002C0220F23
:108D5000331F8A95E2F725830895E82FE695E69577
:108D6000E695F0E0F096A5E0EE0FFF1FAA95E1F77B
:108D7000877021E030E002C0220F331F8A95E2F7AE
:108D8000268308954091CA01E62FF72F8093CA01E8
:108D900084914093CA0108958FEF8093700080936F
:108DA00071008093720080937300809374008093AD
:108DB0007500809376009FB7F89480915000826090
:108DC000809350009FBF8091510081FFFCCF80E4D1
:108DD00090E061E00E94C2489FB7F89480915000F3
:108DE0008E7F809350009FBF0895FC019FB7F89439
:108DF000E059FF4F60958081862380839FBF08954F
:108E0000FC019FB7F894E059FF4F8081862B808347
:108E10009FBF0895AB01282F26952695269530E013
:108E2000205D3F4F877061E070E002C0660F771FE2
:108E30008A95E2F7C90175E0880F991F7A95E1F7E5
:108E40000E949247089580E260E073E00E940A4722
:108E500081E260E073E00E940A4782E260E073E032
:108E60000E940A4783E260E073E00E940A4784E2BE
:108E700060E073E00E940A4785E260E073E00E94D0
:108E80000A4786E260E073E00E940A4787E260E0FA
:108E900073E00E940A4788E168E170E00E940A4797
:108EA00089E168E170E00E940A478AE168E170E0C8
:108EB0000E940A478BE168E170E00E940A478CE15A
:108EC00068E170E00E940A478DE168E170E00E946D
:108ED0000A4788E768E170E00E940A4789E768E18D
:108EE00070E00E940A4788E067E070E00E940A474D
:108EF0008BE060E071E00E940A4783E160E073E08C
:108F00000E940A4782E160E070E00E940A478BE11C
:108F100060E073E00E940A478AE160E070E00E942E
:108F20000A470895CF93DF93DC0120E030E0C62F9D
:108F3000D0E0CE01022E02C0959587950A94E2F703
:108F400080FF04C0FD01E20FF31F408B2F5F3F4FF6
:108F50002830310571F750FF0DC051FF04C0159640
:108F60006C93159703C016966C93169711966C9395
:108F7000119703C012966C931297DF91CF910895C9
:108F80009091020481E092FD80E00895DC01CB0124
:108F9000109200042091010420FDFCCFE0E0F4E0F9
:108FA00080879187A0931334B093143481E0809329
:108FB000000408950F931F932FB7F8940091133472
:108FC000109114348091080490910904009731F4B1
:108FD0003091030430FF02C00F5F1F4F2FBF20E00E
:108FE00030E0980111270027A0E0B0E0082B192BF2
:108FF0002A2B3B2BB801C9011F910F910895DC0169
:10900000CB01E0E0F4E021E0228384879587809320
:10901000173490931834A0931534B0931634E0E0CD
:10902000F4E08091010480FDFACF82E0838385E043
:10903000828308958093193490931A34089580E0C0
:1090400090E064E00E94F54621E0E0E4F0E0238354
:10905000E0E0F4E08FEF9FEF828793871086118620
:109060002283208308951F920F920FB60F9208B6A5
:109070000F9211248F939F93809113349091143405
:10908000019680931334909314349F918F910F9095
:1090900008BE0F900FBE0F901F9018951F920F9251
:1090A0000FB60F9208B60F9209B60F920BB60F9239
:1090B00011240F931F932F933F934F935F936F93BD
:1090C0007F938F939F93AF93BF93EF93FF93009101
:1090D0001334109114344091153450911634041700
:1090E0001507B8F181E0E0E0F4E08283E091193403
:1090F000F0911A34309769F1809108049091090435
:1091000020E030E0980111270027A0E0B0E0082B14
:10911000192B2A2B3B2BCA01A0E0B0E0DC019927D8
:109120008827409117345091183460E070E0842B08
:10913000952BA62BB72B80179107A207B30730F00A
:109140008C019D010F5F1F4F2F4F3F4FC901B80189
:109150001995FF91EF91BF91AF919F918F917F9161
:109160006F915F914F913F912F911F910F910F90B0
:109170000BBE0F9009BE0F9008BE0F900FBE0F9050
:109180001F9018951BBEFC0128ED24BF6083089535
:1091900022E08030920771F480915F33982F9F5FB7
:1091A00090935F338823B9F481E090E062E00E94FD
:1091B000F546089522E08034920769F48091603387
:1091C000982F9F5F90936033882329F482E090E08A
:1091D00062E00E94F546089522E08030920769F42B
:1091E00080915F33815080935F338823B1F481E0B5
:1091F00090E062E00E940047089522E080349207E8
:1092000061F480916033815080936033882329F426
:1092100082E090E062E00E9400470895CF93DF93E0
:1092200081309105C1F08130910520F082309105A7
:1092300079F51DC082E061E270E00E94C246C82F4D
:1092400082E060E270E00E94C2463C2F20E090E0A5
:10925000822B932B1FC082E065E270E00E94C24621
:10926000D82F80E0C82F82E064E270E00BC082E07B
:109270006FE270E00E94C246D82F80E0C82F82E0E3
:109280006EE270E00E94C24690E08C2B9D2B02C0E3
:1092900080E090E0DF91CF9108951F920F920FB67A
:1092A0000F9208B60F9209B60F920BB60F921124C7
:1092B0002F933F934F935F936F937F938F939F93DE
:1092C000AF93BF93EF93FF93E0E0F2E044A155A189
:1092D000E0915B33F0915C3380E092E061E01995BE
:1092E000FF91EF91BF91AF919F918F917F916F917E
:1092F0005F914F913F912F910F900BBE0F9009BE40
:109300000F9008BE0F900FBE0F901F9018951F92E0
:109310000F920FB60F9208B60F9209B60F920BB6C6
:109320000F9211242F933F934F935F936F937F93EB
:109330008F939F93AF93BF93EF93FF93E0E0F2E09F
:1093400044A555A5E0915B33F0915C3380E092E059
:1093500062E01995FF91EF91BF91AF919F918F912D
:109360007F916F915F914F913F912F910F900BBE25
:109370000F9009BE0F9008BE0F900FBE0F901F9068
:1093800018951F920F920FB60F9208B60F9209B65A
:109390000F920BB60F9211242F933F934F935F932D
:1093A0006F937F938F939F93AF93BF93EF93FF93AD
:1093B000E0E0F2E044A955A9E0915B33F0915C3321
:1093C00080E092E064E01995FF91EF91BF91AF9139
:1093D0009F918F917F916F915F914F913F912F91CD
:1093E0000F900BBE0F9009BE0F9008BE0F900FBEDE
:1093F0000F901F9018951F920F920FB60F9208B6FC
:109400000F9209B60F920BB60F9211242F933F9330
:109410004F935F936F937F938F939F93AF93BF937C
:10942000EF93FF93E0E0F2E044AD55ADE0915B33A4
:10943000F0915C3380E092E068E01995FF91EF9144
:10944000BF91AF919F918F917F916F915F914F915C
:109450003F912F910F900BBE0F9009BE0F9008BE49
:109460000F900FBE0F901F9018951F920F920FB67E
:109470000F9208B60F9209B60F920BB60F921124F5
:109480002F933F934F935F936F937F938F939F930C
:10949000AF93BF93EF93FF93E0E4F2E044A155A1B3
:1094A000E0915D33F0915E3380E492E061E01995E4
:1094B000FF91EF91BF91AF919F918F917F916F91AC
:1094C0005F914F913F912F910F900BBE0F9009BE6E
:1094D0000F9008BE0F900FBE0F901F9018951F920F
:1094E0000F920FB60F9208B60F9209B60F920BB6F5
:1094F0000F9211242F933F934F935F936F937F931A
:109500008F939F93AF93BF93EF93FF93E0E4F2E0C9
:1095100044A555A5E0915D33F0915E3380E492E07F
:1095200062E01995FF91EF91BF91AF919F918F915B
:109530007F916F915F914F913F912F910F900BBE53
:109540000F9009BE0F9008BE0F900FBE0F901F9096
:1095500018951F920F920FB60F9208B60F9209B688
:109560000F920BB60F9211242F933F934F935F935B
:109570006F937F938F939F93AF93BF93EF93FF93DB
:10958000E0E4F2E044A955A9E0915D33F0915E3347
:1095900080E492E064E01995FF91EF91BF91AF9163
:1095A0009F918F917F916F915F914F913F912F91FB
:1095B0000F900BBE0F9009BE0F9008BE0F900FBE0C
:1095C0000F901F9018951F920F920FB60F9208B62A
:1095D0000F9209B60F920BB60F9211242F933F935F
:1095E0004F935F936F937F938F939F93AF93BF93AB
:1095F000EF93FF93E0E4F2E044AD55ADE0915D33CD
:10960000F0915E3380E492E068E01995FF91EF916C
:10961000BF91AF919F918F917F916F915F914F918A
:109620003F912F910F900BBE0F9009BE0F9008BE77
:109630000F900FBE0F901F9018951F93CF93DF933D
:10964000EC011FB7F8940E94C84888818160888324
:109650001FBFDF91CF911F910895CF93CFB7F8949B
:10966000FC0120812E7F20830E94EC48CFBFCF9148
:10967000089522E08030920721F481E090915F33D9
:1096800007C022E08034920739F481E09091603382
:10969000992319F480E0089580E00895DF92EF9215
:1096A000FF920F931F93CF93DF93EC018B0182E026
:1096B000C030D80719F480E090E006C0E2E0C03482
:1096C000DE0721F581E090E00E940E497C01DFB6C3
:1096D000F894CE010E94C848288182E08883EC86F5
:1096E000FD86F80185819681888F998F82818A8392
:1096F00084818C8383818B838181898321708081A4
:10970000282B2883CE010E94EC48DFBEDF91CF9149
:109710001F910F91FF90EF90DF900895FF920F93AC
:109720001F93CF93DF93EC018B01FFB6F8940E9457
:10973000C8488881807CF8018083888D998D8583D5
:1097400096838A8182838C8184838B8183838981C0
:109750008183CE010E94EC48FFBEDF91CF911F9123
:109760000F91FF900895DF92EF92FF920F931F9356
:10977000CF93DF937C018A01862F90E083709070F5
:10978000009721F46695669582E001C080E060FF55
:109790008F5FE701A09690E023E0880F991F2A953C
:1097A000E1F7C80FD91FDFB6F894C7010E94C84877
:1097B000F8018081888382818A8381818983C701BE
:1097C0000E94EC48DFBEDF91CF911F910F91FF9077
:1097D000EF90DF900895DF92EF92FF920F931F9327
:1097E000CF93DF937C018A01862F90E08370907085
:1097F000009721F46695669582E001C080E060FFE5
:109800008F5FE701A09690E033E0880F991F3A95AB
:10981000E1F7C80FD91FDFB6F894C7010E94C84806
:109820008881F80180838A81828389818183C7014D
:109830000E94EC48DFBEDF91CF911F910F91FF9006
:10984000EF90DF9008952FB7F89432E080309307BF
:1098500029F460935B3370935C3308C032E080344A
:10986000930721F460935D3370935E332FBF0895A7
:109870008091CF0187FDFCCF08951F93CF93DF9395
:10988000C0ECD1E01A858A878BEC91E061E00E9400
:10989000C2481A87DF91CF911F910895682F82E007
:1098A00070E00E94C2460895CF93DF93EC0188E0F8
:1098B0000E944E4C888389E00E944E4C89838AE046
:1098C0000E944E4C8A838BE00E944E4C8B838CE02E
:1098D0000E944E4C8C838DE00E944E4C8D8380E123
:1098E0000E944E4C8E8382E10E944E4C8F8383E116
:1098F0000E944E4C888784E10E944E4C898785E106
:109900000E944E4C8A87DF91CF9108950F931F9349
:10991000CF93DF930F920F92CDB7DEB789839A83EF
:109920000E94384C00EC11E0F80112829A81918378
:109930008981808386E090E00E943D4CF80184811B
:109940000F900F90DF91CF911F910F910895EF929B
:10995000FF920F931F93CF93DF9300D00F92CDB759
:10996000DEB77C01CB014B835C8369839A830E94C1
:10997000384C0CEC11E0F801208128602083B701FD
:109980006050704F89819A814B815C810E9488541C
:10999000F8018081877F80832496CDBFDEBFDF9171
:1099A000CF911F910F91FF90EF9008950E94384C36
:1099B0008091CF0181FF09C086E3E0ECF1E082876E
:1099C0008BEC91E061E00E94C2480895EF92FF9213
:1099D0001F93CF93DF9300D0CDB7DEB720ECE22EFC
:1099E00021E0F22EF701128569838A839B830E940E
:1099F000D64C0E94384C23E3F701228712829B81C8
:109A000091838A8180836981648385E382878BEC7B
:109A100091E061E00E94C248F70112872396CDBF12
:109A2000DEBFDF91CF911F91FF90EF900895EF92ED
:109A3000FF921F93CF93DF930F920F92CDB7DEB7B4
:109A400030ECE32E31E0F32EF70112856A8389832F
:109A50000E94384C93E3F701928712821182898128
:109A600080836A81648312870F900F90DF91CF917A
:109A70001F91FF90EF900895FF920F931F93CF9344
:109A8000DF93EC0100EC11E0F090CA010E94384C29
:109A900083E3F80182871282118280E08093C00103
:109AA000999194838F5F8032C9F7E0ECF1E0F28600
:109AB000DF91CF911F910F91FF900895CF93DF9386
:109AC0000F92CDB7DEB789830E94384C898190E030
:109AD00045E0880F991F4A95E1F7E0ECF1E012822A
:109AE0009183808385E390E00E943D4C0F90DF914D
:109AF000CF910895CF92DF92EF92FF920F931F9331
:109B0000CF93DF938C016B017A012BC0C8018F7159
:109B100090700097D1F480E2E816F104B0F0C6012D
:109B20000E943C4DC80155E0969587955A95E1F7FE
:109B30000E945E4D005E1F4FE0E2F0E0CE0EDF1EA1
:109B400080EE9FEFE80EF91E0CC0E8012196C801D7
:109B5000F60161916F010E94E64C0894E108F1085A
:109B60008E01E114F10491F6DF91CF911F910F91D5
:109B7000FF90EF90DF90CF900895CF93DF930F92F7
:109B8000CDB7DEB789830E94384C898190E065E0CB
:109B9000880F991F6A95E1F7E0ECF1E0128291835A
:109BA000808384E390E00E943D4C0F90DF91CF9141
:109BB0000895EF92FF921F93CF93DF930F92CDB74B
:109BC000DEB770ECE72E71E0F72E1091CA018983A1
:109BD0000E94D64C0E94384C93E3D7011A969C936E
:109BE0001A9712961C92129711961C92119790E058
:109BF000E0ECF1E089819093C00184839F5F903213
:109C0000D1F7E0ECF1E012870F90DF91CF911F9137
:109C1000FF90EF900895CF93DF930F92CDB7DEB70B
:109C200089830E94384C898190E0E5E0880F991F74
:109C3000EA95E1F7E0ECF1E012829183808382E320
:109C400090E00E943D4C0F90DF91CF910895CF930B
:109C5000C82F8FEF0E94D94D8C2F0E940B4ECF91B1
:109C600008950E94384C80E390E00E943D4C089596
:109C70008FEF0E94D94D0E94314E0895CF92DF920E
:109C8000EF92FF921F93CF93DF936B017C01DA0178
:109C9000C901C0ECD1E01A852AE32A87C882772758
:109CA0006F2D5E2D4D2D49836701EE24FF24CA825E
:109CB0008C83492F5A2F6B2F77274D83CD01AA27ED
:109CC000BB278E838BEC91E061E00E94C2481A872B
:109CD000DF91CF911F91FF90EF90DF90CF9008958B
:109CE000CF92DF92EF92FF920F931F93CF93DF9368
:109CF0000F920F92CDB7DEB7F82EE92E8A016901D7
:109D000069837A830E94384C6981862F7A81972FE4
:109D1000AF2DBE2D0EC00BB6ABBFFC0127910BBE05
:109D2000F80121938F010196A11DB11D0894C1086E
:109D3000D108C114D10479F70F900F90DF91CF9122
:109D40001F910F91FF90EF90DF90CF900895EF92C9
:109D5000FF920F931F93CF93DF93DC01CB017A0126
:109D60008901EC01D1700AC081E0BE010E94C246A7
:109D7000F70181937F0121960150104001151105D3
:109D800099F7DF91CF911F910F91FF90EF90089578
:109D90002F923F924F925F926F927F928F929F92FB
:109DA000AF92BF92CF92DF92EF92FF920F931F93E9
:109DB000CF93DF930F920F92CDB7DEB7DC01CB01CB
:109DC0002A017901702E8C01662457C061E0C62EED
:109DD000D12C8824992454011401772089F081E042
:109DE000B4010E94C246898381E0B6010E94C24646
:109DF0008A8389819A812FEF8F3F920731F407C0C0
:109E00008FEF9FEF89839A8302C066246394E114E5
:109E1000F104D9F00215130561F40894E108F10882
:109E20000F5F1F4FD2018D912D018983E114F10441
:109E300061F00C151D0549F40894E108F1080F5F65
:109E40001F4FF20181912F018A8349815A81C501F7
:109E5000B4010E94870782E090E0A0E0B0E0880EA5
:109E6000991EAA1EBB1EA2E0B0E0CA0EDB1EB1E026
:109E7000CB16B2E0DB0609F0AFCFE114F10409F034
:109E8000A5CF662041F00E94384C60E070E0CB0125
:109E900048E10E9478070E94384C60E070E0CB01F6
:109EA0004AE10E9478070F900F90DF91CF911F91A8
:109EB0000F91FF90EF90DF90CF90BF90AF909F9069
:109EC0008F907F906F905F904F903F902F9008956C
:109ED0002F923F924F925F926F927F928F929F92BA
:109EE000AF92BF92CF92DF92EF92FF920F931F93A8
:109EF000CF93DF9300D000D0CDB7DEB7DC01CB012C
:109F00004B835C831901412CEEEF5E2EEFEF6E2E3A
:109F1000EFEF7E2E482259226A227B226C017D01BE
:109F20007AC00E94384C5301420120E031E010E039
:109F3000002369F00BB6ABBEF401879196910BBE7E
:109F400089839A834FEF8F3F940731F406C08FEFD8
:109F50009FEF89839A8301C011E02114310471F1CC
:109F6000C814D904EA04FB0489F4089421083108D0
:109F70000894C11CD11CE11CF11CAB81BC818D91EA
:109F8000AB83BC83898321143104C1F0D501C401A2
:109F90000196A11DB11DC816D906EA06FB0671F48B
:109FA0000894210831080894C11CD11CE11CF11C43
:109FB000EB81FC818191EB83FC838A8349815A8107
:109FC000C501B4012D833E830E94870782E090E0A3
:109FD000A0E0B0E0880E991EAA1EBB1E2D813E8116
:109FE0002150304009F0A4CF112331F00E94384CA9
:109FF000C301B20145E205C00E94384CC301B20161
:10A0000044E20E94780780E092E0A0E0B0E0480ED1
:10A01000591E6A1E7B1E2114310409F082CF269638
:10A02000CDBFDEBFDF91CF911F910F91FF90EF90D9
:10A03000DF90CF90BF90AF909F908F907F906F9068
:10A040005F904F903F902F9008950F931F93CF9361
:10A05000DF930F92CDB7DEB789830E94384C00ECB6
:10A0600011E08981F801808387E090E00E943D4CF7
:10A07000F80184810F90DF91CF911F910F91089586
:10A08000629FD001739FF001829FE00DF11D649FDC
:10A09000E00DF11D929FF00D839FF00D749FF00D68
:10A0A000659FF00D9927729FB00DE11DF91F639F09
:10A0B000B00DE11DF91FBD01CF0111240895991BB9
:10A0C00079E004C0991F961708F0961B881F7A95AF
:10A0D000C9F78095089597FB092E07260AD077FDCA
:10A0E00004D049D006D000201AF4709561957F4FB6
:10A0F0000895F6F7909581959F4F0895A1E21A2E45
:10A10000AA1BBB1BFD010DC0AA1FBB1FEE1FFF1F1B
:10A11000A217B307E407F50720F0A21BB30BE40B6B
:10A12000F50B661F771F881F991F1A9469F76095B2
:10A130007095809590959B01AC01BD01CF0108956C
:10A1400097FB092E05260ED057FD04D0D7DF0AD085
:10A15000001C38F450954095309521953F4F4F4F56
:10A160005F4F0895F6F790958095709561957F4FB4
:10A170008F4F9F4F0895AA1BBB1B51E107C0AA1F19
:10A18000BB1FA617B70710F0A61BB70B881F991F98
:10A190005A95A9F780959095BC01CD010895CF936C
:10A1A000DF93AC018230910510F442E050E0E09181
:10A1B0001D34F0911E3420E030E0A0E0B0E024C077
:10A1C0008081918184179507D0F08417950771F4E9
:10A1D00082819381109729F012968D939C93139707
:10A1E0002CC080931D3490931E3427C02115310557
:10A1F00019F08217930718F49C01BD01EF019281B9
:10A200008381DF01E92FF82F3097D1F62115310531
:10A21000F9F0C901841B950B8430910580F48A8183
:10A220009B816115710521F0FB018283938304C03A
:10A2300080931D3490931E34FE01329642C0FE017D
:10A24000E80FF91F4193519302978883998339C08E
:10A2500080911B3490911C34009741F48091FC3123
:10A260009091FD3180931B3490931C342091FA31EE
:10A270003091FB312115310541F42DB73EB7809166
:10A28000FE319091FF31281B390BE0911B34F09186
:10A290001C34E217F30798F42E1B3F0B24173507E5
:10A2A00070F0CA0102962817390748F08E0F9F1FD9
:10A2B00080931B3490931C344193519302C0E0E08F
:10A2C000F0E0CF01DF91CF9108950F931F93CF93CB
:10A2D000DF939C01009709F48CC0DC011297129661
:10A2E0001D921C92139760911D3470911E3461155C
:10A2F000710589F48D919C911197820F931F209184
:10A300001B3430911C342817390769F5A0931B348E
:10A31000B0931C346EC0FB0140E050E001C0FC0172
:10A32000EA17FB0730F482819381AF010097B9F7F8
:10A330001FC0E9012297EA83FB8308811981C901C3
:10A34000800F911F8E179F0759F480819181800F94
:10A35000911F029688839983828193818A839B834C
:10A360004115510529F4A0931D34B0931E3441C00A
:10A37000FA01A283B383C191D191EC0FFD1FAE17F7
:10A38000BF0781F4F901929182918C0F9D1F029673
:10A39000DA018D939C9311978281938112968D930C
:10A3A0009C931397E0E0F0E002C0FB01BC01DB01ED
:10A3B00012968D919C9113970097B9F7CB01029655
:10A3C0002D913C911197820F931F20911B34309156
:10A3D0001C342817390769F4309729F410921D347A
:10A3E00010921E3402C01282138260931B34709349
:10A3F0001C34DF91CF911F910F9108958F929F92FE
:10A40000AF92BF92CF92DF92EF92FF920F931F9382
:10A41000CF93DF930F920F92CDB7DEB78C010097E9
:10A4200029F4CB010E94CF508C01B8C0DC01A60FEB
:10A43000B71FFC013297AE17BF0708F4ADC02081EB
:10A44000318126173707B0F02530310508F4A6C052
:10A45000C90104978617970708F4A0C0225030401E
:10A46000261B370B2D933D93CD01608371830E9492
:10A47000655194C06B01C21AD30A5C01A20EB31ECF
:10A48000E0911D34F0911E3440E050E0882499247E
:10A4900049C0EA15FB05E1F5E080F180C7010296AD
:10A4A0008C159D05A8F1A7014C195D09CA010296FA
:10A4B0000F2EFEEFCF2EFFEFDF2EF02DC00ED11EA0
:10A4C0008530910578F08281938112968D939C93CB
:10A4D00013974D935C931197F601608371839A2FC4
:10A4E0008B2F0AC0C90102968E0D9F1DD6018D9338
:10A4F0009C931197928183818114910421F0F4013E
:10A50000928383834BC090931D3480931E3446C046
:10A51000808191814817590708F4AC0182819381A9
:10A520004F01FC01309709F0B4CF80911B3490911A
:10A530001C348A159B05E9F446175707D0F480911F
:10A54000FA319091FB31009741F48DB79EB720917D
:10A55000FE313091FF31821B930BA817B907E0F44D
:10A56000A0931B34B0931C34F8013297608371833D
:10A5700015C0CB0129833A830E94CF507C012981E9
:10A580003A81009749F0B801A9010E948854C80196
:10A590000E946551870102C000E010E0C8010F90E1
:10A5A0000F90DF91CF911F910F91FF90EF90DF906F
:10A5B000CF90BF90AF909F908F9008952F923F9231
:10A5C0004F925F926F927F928F929F92BF92CF92A3
:10A5D000DF92EF92FF920F931F93CF93DF933B0194
:10A5E0008A016115710519F0FB01808391830115C2
:10A5F000110539F09801225030402332310508F01E
:10A6000003C16C0176010894C11CD11CF701C08103
:10A6100046018C2F90E00E943954009799F7CD3273
:10A6200049F4F701C181B2E08B2E912C8E0C9F1C56
:10A63000D1E00AC0CB3239F4F701C181A2E08A2E01
:10A64000912C8E0C9F1CD0E00115110519F00031E2
:10A650001105C1F4C03381F4F4018081883711F011
:10A66000883551F4F401C18182E090E0880E991E92
:10A67000D26000E110E006C00115110519F4C033E5
:10A68000C1F422C008301105F9F00930110524F495
:10A690000230110509F507C00A30110551F00031EB
:10A6A0001105D1F427C0C12CD12CE12C70E4F72E78
:10A6B00026C00AE010E06CECC62E6CECD62E6CECDA
:10A6C000E62E6CE0F62E1BC008E010E0C12CD12C69
:10A6D000E12C50E1F52E13C09801442737FD409539
:10A6E000542F60E070E080E090E80E947E506901A5
:10A6F0007A0105C0C12CD12CE12C48E0F42E20E0D9
:10A7000040E050E0BA011801442437FC4094542C36
:10A7100030EDB32EBC0E99E09B1570F48C2F815454
:10A720008A3118F499ECB92E06C08C2F81568A31E3
:10A7300050F589EAB82EBC0E8B2D90E0801791075A
:10A7400014F527FD1CC0C416D506E606F706A0F0D2
:10A75000CB01BA01A20191010E944050AB01BC01A2
:10A760004B0D511D611D711D4130E0E05E07E0E0C1
:10A770006E07E0E87E0710F02FEF01C021E0F40142
:10A78000C1914F01C5CF6114710489F0222339F0C2
:10A79000089481089108F3018082918208C0D1FF5A
:10A7A0001AC0C4010297F3018083918314C027FF6C
:10A7B00012C0D0FF05C040E050E060E070E804C087
:10A7C0004FEF5FEF6FEF7FE782E290E080931F34FF
:10A7D0009093203416C0D0FF08C0709560955095B6
:10A7E00041955F4F6F4F7F4F0CC077FF0AC082E2E9
:10A7F00090E080931F34909320344FEF5FEF6FEF22
:10A800007FE78A019B0103C000E010E09801B801D6
:10A81000C901DF91CF911F910F91FF90EF90DF90D1
:10A82000CF90BF909F908F907F906F905F904F9050
:10A830003F902F900895FC0188279927E894219153
:10A840002032E9F3293010F02E30C8F32B3241F0DA
:10A850002D3239F4689404C00E946455820F911D12
:10A86000219120532A30C0F31EF4909581959F4F7B
:10A870000895911182C6803219F089508550D0F721
:10A880000895FB01DC0102C005900D92415050403B
:10A89000D8F70895FC0105900020E9F78095909580
:10A8A0008E0F9F1F08950F931F93CF93DF930F92E7
:10A8B0000F92CDB7DEB7BC01DC010D900020E9F7A7
:10A8C000CD01861B970B69837A830E94CF508C0140
:10A8D00069817A81009711F00E94DC54C8010F90C1
:10A8E0000F90DF91CF911F910F9108954EE253E3A6
:10A8F0000E943D550895FB01DC0104C08D9101903B
:10A90000801921F441505040C8F7881B990B0895D5
:10A91000FB01DC0102C001900D9241505040D8F77C
:10A9200008956817790768F4FB01DC01E40FF51F4F
:10A93000A40FB51F02C002900E9241505040D8F7AC
:10A9400008950C948854DC0101C06D93415050402F
:10A95000E0F70895FB01DC018D9181341CF08B350B
:10A960000CF4805E619161341CF06B350CF4605E18
:10A97000861B611189F3990B0895FB01DC010D9091
:10A980000020E9F7119701900D920020E1F708955A
:10A99000FC018191861721F08823D9F79927089522
:10A9A0003197CF010895FB01DC018D910190801951
:10A9B0000110D9F3990B0895FB01DC0101900D9270
:10A9C0000020E1F70895FB01DC014150504088F080
:10A9D0008D9181341CF08B350CF4805E6191613473
:10A9E0001CF06B350CF4605E861B611171F3990BE2
:10A9F0000895881BFCCFFB01DC014150504030F032
:10AA00008D910190801919F40020B9F7881B990BDA
:10AA10000895FB01DC014150504048F001900D9237
:10AA20000020C9F701C01D9241505040E0F7089541
:10AA3000FC0181E090E00190061609F4CF010020AE
:10AA4000D1F701970895FB0151915523A9F0BF015A
:10AA5000DC014D9145174111E1F759F4CD01019009
:10AA6000002049F04D9140154111C9F3FB014111FE
:10AA7000EFCF81E090E001970895FA01A191B081B4
:10AA8000009719F41097E1F0CD01DC01CD010D9094
:10AA9000002011F4C00113C0FB012191222319F001
:10AAA0002015D9F7F3CFFB012191201519F41E923F
:10AAB000119606C02223C1F70D900020A1F7D00106
:10AAC000FA01A193B08308957AE0979F902D879F14
:10AAD000802D910D112408950F931F93CF93DF9331
:10AAE000CDB7DEB72E97CDBFDEBF0E891F89888D0B
:10AAF000998D26E02C8309831A8397FF02C080E09A
:10AB000090E801978D839E83AE01445E5F4FCE0136
:10AB100001966A8D7B8D0E94F1554D815E8157FDB6
:10AB20000AC02F813885421753070CF49A01020F8F
:10AB3000131FF80110822E96CDBFDEBFDF91CF919B
:10AB40001F910F910895CF93DF93CDB7DEB72E9766
:10AB5000CDBFDEBF85E08C838C899D8989839A83F4
:10AB6000AE01485E5F4FCE0101966E897F890E94DB
:10AB700090592E96CDBFDEBFDF91CF9108950F93F0
:10AB80001F93CF93DF93CDB7DEB72E97CDBFDEBF38
:10AB90008C0186E08C8309831A8377FF02C060E012
:10ABA00070E8615070406D837E83CE010196BA01DA
:10ABB000A9010E94F1554D815E8157FD0AC02F8188
:10ABC0003885421753070CF49A01020F131FF8013E
:10ABD00010822E96CDBFDEBFDF91CF911F910F91D6
:10ABE00008952F923F924F925F926F927F928F9231
:10ABF0009F92AF92BF92CF92DF92EF92FF920F930C
:10AC00001F93CF93DF93CDB7DEB72D97CDBFDEBFB8
:10AC10003C016C877D875A01FC0116821782838173
:10AC200081FFC8C12E010894411C511CF30193817E
:10AC3000EC85FD8593FD859193FF8191EC87FD87E0
:10AC4000882309F4B3C1853241F493FD859193FFC4
:10AC50008191EC87FD87853229F490E0B3010E9451
:10AC6000215BE4CFFF24EE2410E01032B0F48B32ED
:10AC700069F08C3228F4803251F0833271F40BC0C9
:10AC80008D3239F0803349F411602CC012601460A9
:10AC900029C0186027C0106125C017FD2EC0282FBD
:10ACA00020532A3098F416FF08C08F2D880FF82EF5
:10ACB000FF0CFF0CF80EF20E15C08E2D880FE82E3B
:10ACC000EE0CEE0CE80EE20E10620CC08E3221F497
:10ACD00016FD6CC1106406C08C3611F4106802C0F9
:10ACE000883659F4EC85FD8593FD859193FF81911C
:10ACF000EC87FD87882309F0B8CF982F95549330BF
:10AD000018F09052933038F424E030E0A20EB31ED5
:10AD10003FE339830FC0833631F0833781F08335C9
:10AD200009F05AC022C0F5018081898322E030E019
:10AD3000A20EB31E21E0C22ED12C420114C092E01B
:10AD4000292E312C2A0C3B1CF5018080918016FFA6
:10AD500003C06F2D70E002C06FEF7FEFC4010E944F
:10AD6000D65A6C0151011F7715C082E0282E312C74
:10AD70002A0C3B1CF5018080918016FF03C06F2DCB
:10AD800070E002C06FEF7FEFC4010E94CB5A6C01EC
:10AD90001068510113FD1CC006C080E290E0B301B1
:10ADA0000E94215BEA948E2D90E0C816D906A8F384
:10ADB0000FC0F40117FD859117FF81914F0190E0BD
:10ADC000B3010E94215BE110EA940894C108D10804
:10ADD000C114D10471F7E7C0843611F0893651F5FA
:10ADE000F50117FF07C080819181A281B38124E022
:10ADF00030E008C080819181AA2797FDA095BA2FE5
:10AE000022E030E0A20EB31E012F0F76B7FF08C07C
:10AE1000B095A095909581959F4FAF4FBF4F00681B
:10AE2000BC01CD01A2012AE030E00E946A5BD82E6D
:10AE3000D4183FC0853721F41F7E2AE030E020C0BF
:10AE4000197F8F36A9F0803720F4883509F0AEC01D
:10AE50000BC0803721F0883709F0A8C001C010610D
:10AE600014FF09C0146007C014FF08C0166006C0B4
:10AE700028E030E005C020E130E002C020E132E00F
:10AE8000F50117FF07C0608171818281938144E0E1
:10AE900050E006C06081718180E090E042E050E0C7
:10AEA000A40EB51EA2010E946A5BD82ED418012FF1
:10AEB0000F7706FF09C00E7FDF1430F404FF06C0D1
:10AEC00002FD04C00F7E02C01D2D01C01F2D802F6A
:10AED00090E004FF0CC0FE01ED0DF11D2081203338
:10AEE00011F4097E09C002FF06C01E5F05C0867806
:10AEF0009070009709F01F5F802E992403FD12C007
:10AF000000FF0DC0FD2C1E1550F4FE0CF11A1E2D75
:10AF100006C080E290E0B3010E94215B1F5F1E1516
:10AF2000C0F304C01E1510F4E11A01C0EE2484FE23
:10AF30000FC080E390E0B3010E94215B82FE1FC03E
:10AF400081FE03C088E590E010C088E790E00DC066
:10AF5000C40186789070009791F081FC02C080E275
:10AF600001C08BE207FD8DE290E0B3010E94215BFE
:10AF700006C080E390E0B3010E94215BFA94DF14E5
:10AF8000C0F3DA94F201ED0DF11D808190E0B30180
:10AF90000E94215BDD20A9F706C080E290E0B301AA
:10AFA0000E94215BEA94EE20C1F740CEF301868136
:10AFB000978102C08FEF9FEF2D96CDBFDEBFDF914F
:10AFC000CF911F910F91FF90EF90DF90CF90BF90A6
:10AFD000AF909F908F907F906F905F904F903F9039
:10AFE0002F90089520FD09C0FC0123FD05C022FF1C
:10AFF00002C073836283518340830895CF92DF92AE
:10B00000EF92FF926B017C0144FD10C046FD10C021
:10B01000D601F701AA0FBB1FEE1FFF1F1094D1F737
:10B02000CA0EDB1EEE1EFF1E81E003C083E001C0DE
:10B0300084E0CC0CDD1CEE1CFF1C8150D1F7C20E4D
:10B04000D11CE11CF11CB601C701FF90EF90DF900D
:10B05000CF9008950F931F93CF93DF938C01C80176
:10B060000E94E15AEC0197FD08C00E9439540097F4
:10B07000B1F7CE01B8010E944D5BCE01DF91CF91B7
:10B080001F910F910895AF92BF92CF92DF92EF92EE
:10B09000FF920F931F93CF93DF938C01D62F5A010A
:10B0A000C22F0E94E15A8B3219F08D3249F4C068E8
:10B0B000D15009F461C0C8010E94E15A97FD5CC0FB
:10B0C000CD7F2C2F2073D1F48033C1F4D15009F4FB
:10B0D0003EC0C8010E94E15A97FD39C0C26088375E
:10B0E00011F0883549F4C064D15089F1C8010E943B
:10B0F000E15A97FF03C02BC0C6FFC061CC24DD24FA
:10B100007601282F2053283080F0C4FD09C02A3052
:10B1100060F0C6FF05C02F7D322F3151363020F050
:10B12000B8010E944D5B10C02750C701B6014C2FDB
:10B130000E94FE576B017C01C260D15059F0C801DA
:10B140000E94E15A97FFDDCFC1FD04C015C0CC2499
:10B15000DD247601C7FF08C0F094E094D094C09439
:10B16000C11CD11CE11CF11CC501B701A6012C2F8B
:10B170000E94F25781E001C080E0DF91CF911F91E2
:10B180000F91FF90EF90DF90CF90BF90AF90089518
:10B190004F925F926F927F928F929F92AF92BF92E7
:10B1A000CF92DF92EF92FF920F931F93CF93DF9393
:10B1B000CDB7DEB7A097CDBFDEBF5C01062F7A0109
:10B1C0006901FE01319680E2DF011D928A95E9F75F
:10B1D000D50113961C91139760E070E020E040E0E9
:10B1E00030E04F0181E0682E712CF60113FD55917E
:10B1F00013FF51916F01552309F47BC05E3519F49B
:10B200006115710549F1832F90E0861797073CF48B
:10B210005D3551F15D3219F4442301F103C044233B
:10B2200009F4252F852F869586958695F401E80FDC
:10B23000F11D852F8770230102C0440C551C8A958F
:10B24000E2F7808184298083521751F0521710F45D
:10B250005F5FE8CF5150E6CF31E003C041E001C06D
:10B2600040E06F5F7F4FC1CF442319F08E81806231
:10B270008E83332351F0FE013196CE0181962081D9
:10B2800020952193E817F907D1F711E001C010E0EC
:10B29000C5010E94E15A9C0197FD23C086958695C1
:10B2A0008695E1E0F0E0EC0FFD1FE80FF11D408115
:10B2B00050E0C9018770907002C0559547958A95F6
:10B2C000E2F740FD05C0C901B5010E944D5B09C010
:10B2D000E114F10419F0D7012D937D010150B9F665
:10B2E00002C0112331F4E114F10429F0F7011082B6
:10B2F00002C0CC24DD24C601A096CDBFDEBFDF9105
:10B30000CF911F910F91FF90EF90DF90CF90BF9062
:10B31000AF909F908F907F906F905F904F90089527
:10B320005F926F927F928F929F92AF92BF92CF92D5
:10B33000DF92EF92FF920F931F93CF93DF930F92C1
:10B34000CDB7DEB77C015B013A01FC0116821782A2
:10B350009924EFC0812F90E00E943954009721F08A
:10B36000C7010E942A58E5C0153241F4F50103FDDA
:10B37000359103FF31915F01353261F4C7010E94BD
:10B38000E15A97FDE2C0181709F4D3C0B7010E9433
:10B390004D5BDDC03A3241F403FD359103FF31913D
:10B3A0005F015524539401C05524882410C0F2E055
:10B3B0005F2A682D70E080E090E040E20E94FE5736
:10B3C000862EF50103FD359103FF31915F01232F97
:10B3D00020532A3060F351FE03C0882019F4B7C00F
:10B3E00088248A94383619F03C3699F40AC0F5015D
:10B3F00003FD359103FF31915F01383651F4F8E0D8
:10B400005F2A44E0542AF50103FD359103FF319191
:10B410005F01332309F49BC084E99EE0632F70E051
:10B4200039830E94C05A3981009709F490C0852D54
:10B4300050FC08C0F3010081118142E050E0640E2D
:10B44000751E02C000E010E03E3651F4F70146815F
:10B45000578160E070E0C801252D0E94F25769C055
:10B46000333691F481FD02C088248394C7010E9481
:10B47000E15A97FD6AC00115110519F0F801819391
:10B480008F018A9499F753C0C7013B3551F4682D59
:10B49000A80195010E94C8585C01009709F047C0B7
:10B4A00041C039830E942A58398197FD4EC03F36EA
:10B4B00061F1303728F4343629F1393649F52AC09C
:10B4C000333719F0353721F51DC0C7010E94E15A05
:10B4D0006C0197FD11C00E943954009729F0C601F4
:10B4E000B7010E944D5B08C00115110519F0F80164
:10B4F000C1928F018A9449F701151105C1F0F80135
:10B50000108215C0F0E25F2A05C040E1542A02C053
:10B5100050E4552AC701682DA801252D0E944358E3
:10B52000882329F4F7018381807379F410C050FED9
:10B530009394F7010381F50103FD159103FF119128
:10B540005F01112309F006CF02C0992019F0892D5F
:10B5500090E002C08FEF9FEF0F90DF91CF911F918E
:10B560000F91FF90EF90DF90CF90BF90AF909F90A2
:10B570008F907F906F905F90089599278827089506
:10B58000FC010590061621F00020D9F7C0010895AE
:10B590003197CF010895FC01059061507040011072
:10B5A000D8F7809590958E0F9F1F0895FC016150EC
:10B5B000704001900110D8F7809590958E0F9F1FD5
:10B5C0000895CF93DF93EC012B8120FF35C026FF38
:10B5D00009C02F7B2B838E819F8101968E839F8351
:10B5E0008A8128C022FF0FC0E881F98180819927D4
:10B5F00087FD9095009719F420622B831DC031962A
:10B60000E883F98311C0EA85FB85CE01199597FF80
:10B610000BC02B813FEF8F3F930711F480E101C0F6
:10B6200080E2822B8B8308C02E813F812F5F3F4FAA
:10B630002E833F8390E002C08FEF9FEFDF91CF9189
:10B6400008950F931F93CF93DF938C01EB018B81B0
:10B6500081FF1BC082FF0DC02E813F818C819D81A7
:10B660002817390764F4E881F9810193E883F983A5
:10B6700006C0E885F985802F1995009731F48E81F1
:10B680009F8101968E839F8302C00FEF1FEFC80139
:10B69000DF91CF911F910F910895FB01238120FF2E
:10B6A00013C026FD11C03FEF8F3F930781F08283C7
:10B6B000922F90649F7D9383268137812150304063
:10B6C0002683378390E008958FEF9FEF08958FEFE3
:10B6D0009FEF0895FA01AA27283051F1203181F116
:10B6E000E8946F936E7F6E5F7F4F8F4F9F4FAF4F8A
:10B6F000B1E03ED0B4E03CD0670F781F891F9A1F9D
:10B70000A11D680F791F8A1F911DA11D6A0F711D50
:10B71000811D911DA11D20D009F468943F912AE05C
:10B72000269F11243019305D3193DEF6CF01089544
:10B73000462F4770405D4193B3E00FD0C9F7F6CF75
:10B74000462F4F70405D4A3318F0495D31FD40523D
:10B75000419302D0A9F7EACFB4E0A69597958795D3
:10B7600077956795BA95C9F70097610571050895B2
:10B770009B01AC010A2E069457954795379527955E
:10B78000BA95C9F7620F731F841F951FA01D0895F6
:04B79000F894FFCF5B
:10B7940000257320257300252D3230732025730D69
:10B7A4000A006F6B006572720025733B25640D0AF5
:10B7B40000257320256420282573290D0A002020E4
:10B7C40020002573202D2068657864756D70286CC1
:10B7D400656E3D2564293A0D0A0025303478202011
:10B7E40000253032782000257325730D0A000820C7
:10B7F40008000D0A002000636F6D6D616E64206E99
:10B804006F7420666F756E643A25730D0A00257394
:10B814002000256300240068656C70007072696EF6
:10B8240074207468697320696E666F726D617469DF
:10B834006F6E002573202D2068657864756D7028FF
:10B844006C656E3D2564293A0A0D00253034782054
:10B854002000253032782000202020003A200020CB
:10B86400202025730A0D0073756363657373007577
:10B874006E6B6E6F776E00616C72656164792069BE
:10B884006E207573650061626F727465640073790C
:10B894006E63206572726F720063616E63656C65BE
:10B8A400642062792072656D6F74650069676E6FDC
:10B8B4007265640074696D656F75740070726F747D
:10B8C4006F636F6C206572726F720064697361627A
:10B8D4006C65640062757379007265747279206CAA
:10B8E40061746572006261642073697A65006F75C2
:10B8F40074206F662072616E6765006F7065726197
:10B9040074696F6E206E6F7420737570706F7274CB
:10B914006564006E6F207065726D697373696F6E14
:10B9240000696E636F6D70617469626C652074790F
:10B9340070650070617468206E6F7420666F756E38
:10B94400640070617273696E67206572726F720051
:10B95400696E76616C6964207374617465006E6FDE
:10B964007420636F6E6E6563746564006F75742014
:10B974006F66206D656D6F72792F6275666665728C
:10B984007300696E76616C696420706172616D65C3
:10B994007465727300756E6B6E6F776E2066616985
:10B9A4006C7572650073772076657273696F6E3A91
:10B9B40025642E25642E25640D0A00636F6E6E5F68
:10B9C400636220736F636B69643A256420636F6EEE
:10B9D4006E65637465643A25640D0A006F6B003B01
:10B9E40000657272000025733B256425730D0A00FF
:10B9F40075736167653A207363616E205B73736965
:10BA0400645D0D0075736167653A207365745F70DA
:10BA14006F6C6C5F706572696F64203C70657269ED
:10BA24006F6420696E206D733E0D0A007065726943
:10BA34006F642025640D0A0075736167653A20738D
:10BA440065745F686561727462656174203C307C02
:10BA5400313E0D0A0075736167653A207365745F42
:10BA64006C6564203C307C313E0D0A006361707368
:10BA74003A3078253032780D0A00756E6B6E6F7728
:10BA84006E0066772076657273696F6E3A25642E50
:10BA940025642E2564206275696C643A25730D0A49
:10BAA400006877207265766973696F6E3A25730D45
:10BAB4000A00687474705F706F7374004C697374F7
:10BAC400656E696E67206F6E2025733A25642F2595
:10BAD400730D0A0075736167653A2066775F757048
:10BAE4006772616465203C6D6574686F642C2065C1
:10BAF4002E672E2022687474705F706F7374223EF8
:10BB0400205B3C69703E203C706F72743E203C7038
:10BB14006174683E5D0D0A002573202564202800A9
:10BB240069703A257320006D61736B3A25732000A8
:10BB340067773A25732000646E733A2573290D0ADA
:10BB440000706565723A25730D0A00757361676547
:10BB54003A206765745F7065657261646472203C45
:10BB6400736F636B69643E0D0A0073656E64696E7E
:10BB74006720256420627974657320746F202573AF
:10BB84003A25640D0A0077726F74653A2564207251
:10BB9400656D61696E3A25640D0A007573616765A8
:10BBA4003A2073656E64746F203C736F636B6964D1
:10BBB4003E203C69703E203C706F72743E203C64B1
:10BBC400617461202E2E2E3E0D0A0073656E646929
:10BBD4006E672025642062797465730D0A0075739D
:10BBE4006167653A2073656E64203C736F636B69AB
:10BBF400643E203C64617461202E2E2E3E0D0A00AA
:10BC040075736167653A20636C6F7365203C736F6D
:10BC1400636B69643E0D0A0075736167653A20635E
:10BC24006F6E6E656374203C736F636B69643E2052
:10BC34003C69703E203C706F72743E0D0A0075734F
:10BC44006167653A206C697374656E203C736F6339
:10BC54006B69643E205B6261636B6C6F675D0D0AA8
:10BC6400006C697374656E5F636220736F636B69E4
:10BC7400643A25642C20616363657074696E67207F
:10BC84002E2E2E200028636F6E6E656374696F6EAE
:10BC9400206C6F73742900726563765F636220732E
:10BCA4006F636B69643A2564206C656E3A25642081
:10BCB40025730D0A0052580075736167653A206256
:10BCC400696E64203C736F636B69643E203C6970E9
:10BCD4003E203C706F72743E0D0A0073747265618D
:10BCE4006D00646772616D007261770075736167DE
:10BCF400653A20736F636B6574203C73747265617D
:10BD04006D7C646772616D7C7261773E205B7072DA
:10BD14006F746F636F6C5D0D0A0075736167653ACC
:10BD2400207365745F6468637064203C307C313ECA
:10BD34000D0A0025732025642028656E61626C65F8
:10BD4400643A2564290D0A0075736167653A2073A6
:10BD540065745F64686370203C307C313E0D0A007A
:10BD640075736167653A207365745F6970616464B3
:10BD740072203C69703E205B6D61736B5D205B6774
:10BD8400775D205B646E735D0D0A004E2F410025C4
:10BD940073202564000D0A002028257320253032E5
:10BDA400783A253032783A253032783A253032786C
:10BDB4003A253032783A253032782000727373692C
:10BDC4003A25642000727373693A4E2F4120007340
:10BDD4006E723A256400736E723A4E2F4100290D3B
:10BDE4000A0025732025642028253032783A25302E
:10BDF40032783A253032783A253032783A25303262
:10BE0400783A25303278290D0A0075736167653AEE
:10BE1400207365745F6368616E6E656C203C636853
:10BE2400616E6E656C3E0D0A0075736167653A203C
:10BE3400636F6E665F6170203C68696464656E3E22
:10BE4400203C626561636F6E5F696E74766C3E0D53
:10BE54000A00202020202020202020202020202014
:10BE6400203C696E6163745F746D6F3E205B636F29
:10BE7400756E7472795D3E0D0A0058202564202584
:10BE8400642025642025642025640075736167653A
:10BE94003A20636F6E665F7073203C7573655F70E4
:10BEA400735F706F6C6C3E203C70735F747261667C
:10BEB4006669635F74696D656F75743E0D0A002071
:10BEC40020202020202020202020202020203C7002
:10BED400735F64656C61793E203C72785F616C6C61
:10BEE4005F6474696D3E203C6C697374656E5F6950
:10BEF4006E74657276616C3E0D0A007573616765D8
:10BF04003A207365745F7073203C307C313E0D0AB7
:10BF140000257320256420282573290D0A007374D5
:10BF240061006170006164686F630077707300750D
:10BF3400736167653A207365745F6D6F6465203C57
:10BF44007374617C61707C6164686F637C77707307
:10BF54003E0D0A007770613200777061007765707A
:10BF64000075736167653A206C696E6B7570205B50
:10BF7400737369645D205B6B65795D205B776570C5
:10BF84007C7770617C777061325D0D0A0075736136
:10BF940067653A207365745F626175647261746584
:10BFA400203C62617564726174653E205B727473D7
:10BFB4006374735D0D0A006572722025642028661F
:10BFC40061696C656420746F20636F6E6669677560
:10BFD400726520686F73742075617274290D0A008C
:10BFE400494E465241004144484F43006E6F206E13
:10BFF40065747320666F756E640D0A006661696C02
:10C00400656420746F20676574206E6574776F7241
:10C014006B206C6973740D0A004253534944202009
:10C02400202020202020202020202020545950454A
:10C034002020204348205253534920534E5220205D
:10C0440041555448202020202020535349440D0AB0
:10C05400002D2D2D2D2D2D2D2D2D2D2D2D2D2D2D39
:10C064002D2D2D2D2D2D2D2D2D2D2D2D2D2D2D2DFC
:10C074002D2D2D2D2D2D2D2D2D2D2D2D2D2D2D2DEC
:10C084002D2D2D2D2D2D2D2D2D2D2D2D2D2D2D2DDC
:10C094002D2D2D2D2D2D0D0A00253032783A2530E9
:10C0A40032783A253032783A253032783A253032AF
:10C0B400783A25303278202000257320202530322C
:10C0C4006420253032642020002530326420202072
:10C0D400004E2F412020004E4F4E4520202020208E
:10C0E4002000574550202020202020200057504178
:10C0F4002D50534B20202000575041322D50534B8C
:10C10400202000575041202020202020200057507C
:10C114004132202020202020002573006C6F6F6B9B
:10C1240075705F63623A20686F7374206E6F742059
:10C13400666F756E640D0A006C6F6F6B75705F636C
:10C14400622069703A25730D0A0075736167653A58
:10C15400206765745F686F737462796E616D6520C2
:10C164003C646E736E616D653E0D0A007363616EAF
:10C1740000776C705F7363616E2873736964290060
:10C184007365745F706F6C6C5F706572696F640067
:10C19400776C705F7365745F706F6C6C5F706572E1
:10C1A400696F642829007365745F686561727462DD
:10C1B40065617400776C705F7365745F6865617244
:10C1C40074626561742829007365745F6C6564002A
:10C1D400776C705F7365745F6C65642829006765AC
:10C1E400745F66775F63617073007072696E742048
:10C1F4006669726D77617265206361706162696CF2
:10C204006974696573006765745F66775F766572E4
:10C2140073696F6E007072696E74206669726D77EF
:10C224006172652076657273696F6E006765745F0D
:10C2340076657273696F6E007072696E7420636CD8
:10C2440069656E742076657273696F6E0066775FD8
:10C254007570677261646500776C705F66775F758F
:10C26400706772616465286D6574686F642C206101
:10C274006464722C20706F72742C2070617468294D
:10C28400006765745F686F737462796E616D6500D1
:10C29400776C705F6765745F686F737462796E61E1
:10C2A4006D6528646E736E616D6529006765745FE2
:10C2B400706565726164647200776C705F67657441
:10C2C4005F706565726164647228736F636B69641F
:10C2D400290073656E64746F00776C705F73656EAC
:10C2E40064746F28736F636B69642C206461746178
:10C2F4002C2069702C20706F7274290073656E6431
:10C3040000776C705F73656E6428736F636B696428
:10C314002C20646174612900636C6F736500776C11
:10C32400705F636C6F736528736F636B6964290056
:10C33400636F6E6E65637400776C705F636F6E6EAF
:10C3440065637428736F636B69642C2069702C2097
:10C35400706F727429006C697374656E00776C7009
:10C364005F6C697374656E28736F636B69642C20EA
:10C374006261636B6C6F67290062696E6400776C3D
:10C38400705F62696E6428736F636B2C2069702C14
:10C3940020706F72742900736F636B657400776C1F
:10C3A400705F736F636B657428747970652C20708B
:10C3B400726F746F29007365745F646863706400DE
:10C3C400776C705F7365745F6468637064282900B8
:10C3D4006765745F6468637000776C705F67657429
:10C3E4005F646863702829007365745F64686370B0
:10C3F40000776C705F7365745F6468637028656E42
:10C4040061626C6529006765745F69706164647258
:10C4140000776C705F6765745F697061646472282B
:10C4240029007365745F69706164647200776C706D
:10C434005F7365745F6970616464722869702C202D
:10C444006D61736B2C2067772C20646E73290067F1
:10C4540065745F6E6574776F726B00776C705F677D
:10C4640065745F6E6574776F726B282900676574F5
:10C474005F68776164647200776C705F6765745F8E
:10C484006877616464722829007365745F63686106
:10C494006E6E656C00776C705F7365745F63686162
:10C4A4006E6E656C282900636F6E665F617000773D
:10C4B4006C705F636F6E665F6170282900636F6ED6
:10C4C400665F707300776C705F636F6E665F707326
:10C4D4002829007365745F707300776C705F7365EF
:10C4E400745F70732829006765745F6D6F646500FD
:10C4F400776C705F6765745F6D6F6465282900737E
:10C5040065745F6D6F646500776C705F7365745FED
:10C514006D6F64652829006C696E6B646F776E00BB
:10C52400776C705F6C696E6B646F776E2829006C32
:10C53400696E6B757000776C705F6C696E6B75708B
:10C5440028737369642C206B65792C206175746879
:10C5540029007365745F6261756472617465007744
:10C564006C705F7365745F62617564726174652871
:10C574002900726573657400776C705F726573650A
:10C58400742829000D0A0047455420002D2D2D2024
:10C5940025732070696E672073746174697374699C
:10C5A4006373202D2D2D0A0D002564207061636BAB
:10C5B400657473207472616E736D69747465642C30
:10C5C4002025642072656365697665640A0D00251B
:10C5D400642062797465732066726F6D2025733AE6
:10C5E4002069636D705F7365713D25640A0D0025D4
:10C5F400642062797465732066726F6D2025733AC6
:10C604002069636D705F7365713D256420446573B3
:10C6140074696E6174696F6E20486F737420556E0F
:10C62400726561636861626C650A0D00256420624D
:10C63400797465732066726F6D2025733A2069637F
:10C644006D705F7365713D256420547970653A257A
:10C65400640A0D006F6B00657272002D63002D7308
:10C6640000257320256420282573290A0D0075737D
:10C674006167653A2070696E67205B2D63203C63B7
:10C684006F756E743E5D205B2D73203C73697A6513
:10C694003E5D203C69703E0A0D0070696E67000AB9
:10C6A4000D0074746370206572723A256420282525
:10C6B40073290A0D0074746370206F6B3A2025642B
:10C6C4002062797465732070726F63657373656437
:10C6D40020696E20256C75206D732C20256C7520C7
:10C6E4004B422F730A0D0074746370206F6B3A20F1
:10C6F40025642062797465732070726F6365737347
:10C70400656420696E2030206D730A0D002E002DA3
:10C7140070002D6E002D6C002D74002D7200257399
:10C7240020256420282573290A0D0065727200747F
:10C7340074637020636F6E6E6563742025733A258D
:10C7440064206E6275663A2564206275666C656E57
:10C754003A256420736F636B69643A25640A0D009B
:10C7640074746370206C697374656E20706F727476
:10C774003A2564206275666C656E3A2564206C7394
:10C784006F636B69643A25640A0D007573616765AC
:10C794003A2074746370205B2D7472706E6C5D0A41
:10C7A4000D00747463700074746370207468726F25
:10C7B4007567687075742074657374006661696C5C
:10C7C400656420746F20676574206E7470207469CA
:10C7D4006D653A2573282564290A0D006E7470204E
:10C7E40074696D653A20253034642D253032642D0A
:10C7F4002530326420253032643A253032643A25BB
:10C804003032640A0D006F6B00657272002573206C
:10C81400256420282573290A0D0075736167653A1C
:10C82400206E7470203C6E74702D73657276657220
:10C834003E0A0D0000001F003B005A0078009700DC
:10C84400B500D400F300110130014E016D01000068
:10C854001F003C005B0079009800B600D500F4008E
:10C86400120131014F016E016E747000676574200E
:10C874007365727665722074696D652066726F6D7A
:10C88400206E7470004E2F4100253032783A2530E6
:10C8940032783A253032783A253032783A253032B7
:10C8A400783A25303278002F002F3F002F696E64CC
:10C8B40065782E68746D6C3F00746F67676C653DB6
:10C8C4004C45442564002F696E6465782E68746D48
:10C8D4006C002F6C6F676F2E676966006C696E6BF6
:10C8E4005F6362206C696E6B3A25640A0D006669A9
:10C8F400726D77617265207570677261646520631B
:10C904006F6D706C6574650A0D006669726D776190
:10C9140072652075706772616465206661696C6513
:10C92400640A0D00616464725F63622069703A6E28
:10C934006F6E650A0D0068747470642073746F7090
:10C944007065640A0D00616464725F6362206970DB
:10C954003A25730A0D0068747470642073746172EC
:10C964007465640A0D006864776972656C65737335
:10C97400006864776972656C6573733132330000E3
:10C984004E0045004F004D005300000021342000AC
:10C99400FFFFFFFF0000000087207D188C20E720A8
:10C9A400F620FE2009211C2124212C213B21442195
:10C9B400492155215E216B2183219121A321B2219B
:10C9C400C021CE21DC21F2210522DC29DD21E1294F
:10C9D400F0298522002A162A1923242A382A7B239F
:10C9E400402A4E2AB1235A2A762AE023852A9C2AF1
:10C9F4007F21A82ABD2A5F24C82AF12A8532002B68
:10CA04001C2BD125292B422B2D26492B6C2B1B2784
:10CA1400712B882BD9278E2BA02B0F28A82BC62B44
:10CA24006528CD2BE92B6329EE2B072CB9290E2C75
:10CA3400262C362A302C402C6C2A492C582CAA2A15
:10CA4400612C762C1825812C922CE02A9D2CBF2C4D
:10CA54006A2BCB2CDD2C8B2CE82CF92CD82C052D17
:10CA6400172D0D2D1F2D2D2D7A2D352D432D3F2EB8
:10CA74004A2D572D752E602D6F2DBF2E782D872DA5
:10CA84000B2F902D9F2D172FA62DC22DB32FCF2DF9
:10CA9400E22D5E30E82D8E27922795279B270A2FBB
:10CAA40003360A2F1230C0391730D8304C3CDC30F2
:0ECAB40001020307F031F231F431F631F831AE
:00000001FF
